:020000041000EA
:1004000000C00208EB0400100D00000049050010B8
:1004100000000000000000000000000000000000DC
:100420000000000000000000000000004505001072
:100430000000000000000000450500104505001008
:100440004505001045050010450500104505001044
:100450004505001045050010450500104505001034
:100460004505001045050010450500104505001024
:100470004505001045050010450500104505001014
:1004800010B5064C2378002B07D1054B002B02D06A
:10049000044800E000BF0123237010BD00060208DD
:1004A00000000000B0910010044B10B5002B03D0E9
:1004B0000349044800E000BF10BDC0460000000032
:1004C00004060208B09100100230800803D0013009
:1004D0000238FCD1C046C0467047EFF3108072B6B8
:1004E000704780F3108870477047FFF7FDFF72B6C2
:1004F0000E4C0F4DAC4209DA21686268A368043BD8
:1005000002DBC858D050FAE70C34F3E709490A4A2D
:100510000020521A02DD043A8850FCDC07480849E2
:100520000860BFF34F8F06F021FEFEE7BC9100107C
:10053000D4910010000602082410020800000208EE
:1005400008ED00E0FEE7FEE700B504207146084232
:1005500002D0EFF3098001E0EFF30880043005F0EA
:10056000BBFEFEE70300093B0122042B02D9203821
:100570004242424110007047F0B5002517000600C6
:100580002C0089B003930E9B02901B0CDBB20493EA
:100590000E9B00911B0ADBB205930E9BDBB2079307
:1005A000731C069333780193002B08D0009B002B1B
:1005B00022DB029A731C9B1A009A9A421CDA0E9B49
:1005C000DBB2002B00D1B4E0019A9A4200D0AEE039
:1005D000009B002B06DB029A731C9B1A009A934225
:1005E00000DDA4E0B31C7678032D00D9A1E028003B
:1005F00006F09EFE8989637B0198FFF7B3FF002810
:1006000039D1079B019A9342D9D04F4E1100300047
:1006100008F078F9031E08D1049B019A93420BD08D
:10062000059B93426FD133003F33032D23D828001D
:1006300006F07EFE0510233533003E33F5E7002F2C
:1006400006D0039A94425ED23F4A9B1A9B003B55C8
:10065000012510E0621C002F0BD003998A4252D270
:1006600039493C195B1A2178181101431B0121708B
:10067000BB5414000225069E92E7621C002F0BD08B
:1006800003998A423FD230493C195B1A217898106D
:1006900001439B012170BB5414000325EBE7002F9D
:1006A00008D0039A94422ED227493A195B1A11783E
:1006B0000B43137001340025DDE71D00002E22D00E
:1006C000009B002B22DB029B009AEB1A9A421DDA58
:1006D000019BB34217D1009B002B04DD029B009AC3
:1006E000EB1A93420FDC2E786B1C029A9D1A002E97
:1006F00004D0009B002B11DBAB420FDA002F18D087
:100700003B5D002B15D00124644219E03000FFF757
:1007100029FF0028DCD02E780135CFE73000FFF725
:1007200021FF0028EFD0029B5E5D0135DFE7002D41
:10073000E9D1039B9C42E6D2002F01D000233B5518
:10074000200009B0F0BDC046688B0010002210B533
:1007500004001000A15C0B00303B092B09D8303895
:100760000818531C032A03D000011A00042BF1D1EE
:1007700010BD0B00413B052B01D83738F0E70B00CB
:10078000613B052B01D85738EAE70020F0E700006D
:10079000F0B50B7885B0039017004D1C222B17D0B5
:1007A000116000202AE05C2A07D1019A5278002AC1
:1007B000F7D0019A013301320192019A013201927C
:1007C000019A1278222A00D1A7E0002AEBD1E8E7AB
:1007D00001950023F4E72B785C2B11D023700135B1
:1007E0000134019B9D42F6D30023039A2370083302
:1007F000D36013000198029A01301A6105B0F0BD70
:100800006B78662B63D014D82F2B61D007D8222B9E
:100810005ED0484B3D601B6802989847C1E75C2B4F
:1008200056D0622BF5D1082323700134063BED1816
:10083000D7E7722B50D006D86E2BEAD10A2323704B
:100840000134083BF3E7742B48D0752BE1D1019BB1
:100850005B1B052BDDDDA81CFFF778FF364B374A05
:10086000C31806009342D4D90028D2D0344B334A5F
:10087000C318934234D8019AAB1DD31A052BC8DD97
:10088000AB795C2BC5D1EB79752BC2D12800083030
:10089000FFF75CFF284B294AC3189342B9D8294B6C
:1008A000B6021E4080238005800D5B020643F618C9
:1008B0000C23254A96421FD9244A9642A9D83F20A4
:1008C0003040802676420643E670042212E00C2374
:1008D000237001340223AAE70D23F9E70923F7E780
:1008E0007F2804D91A4B98420ED90623E1E7062344
:1008F00001222070A4189AE73F20304080267642DB
:100900000643A6700322F5E73F20802306405B42A2
:100910001E43667086330222ECE7019A501AC01A11
:100920000C4B04301B6898470290041E00D058E717
:1009300037E7C046800002080024FFFFFF030000E5
:100940000028FFFF00FC0F00FFFF0000FFFF10006A
:10095000FF07000084000208002803D00378013B51
:100960001F2B00D970470130F6E70000064B10B589
:100970001B6828209847041E03D02822002107F076
:10098000FEFE200010BDC046840002080849094A46
:10099000002803D1084B0B60084B07E00368002BCD
:1009A00000D1054B0B604368002BF5D013607047F6
:1009B000840002088000020821870010358700109B
:1009C000F8B5802604007600002C00D1F8BDE3685D
:1009D0002768334204D1A068002801D0FFF7F0FF58
:1009E000E3680B4D334204D12069002801D02B6805
:1009F00098478022E3689200134204D1206A0028BD
:100A000001D02B68984720002B6898473C00DBE713
:100A100080000208F0B5040085B00F001600002920
:100A200001D1002013E004226F49380007F08AFF4B
:100A3000002803D10223E360381D08E005226B493A
:100A4000380007F07FFF002803D1E060781D05B073
:100A5000F0BD04226649380007F074FF002806D173
:100A600001230122E3600023A261E361E4E73B7814
:100A7000222B05D1320039002000FFF789FEE6E77E
:100A80002D2B03D01A00303A092A24D800250A2237
:100A900003A93800039508F013F803000398874270
:100AA000BFD05A1C0AD1534A914211D10122514B55
:100AB0005242A261E3610423E360C8E7002B07D13F
:100AC00080221206914203D1802300221B06F0E708
:100AD000A361E161EFE75B2B35D1781CFFF73CFFA9
:100AE000037805005D2B26D00023013D0193009380
:100AF000FFF73CFF009B071E6FD0002B19D0019B16
:100B000018604360681CFFF727FF320001003800BF
:100B1000FFF780FFFFF720FF051E06D0037801973F
:100B20002C2BE5D05D2B08D030600098FFF748FFF4
:100B300077E70090E6E7002300931023E360009B33
:100B4000681CA36083E77B2B4BD1781CFFF704FF65
:100B5000037807007D2B38D00023013F01930093D9
:100B6000FFF704FF009B051E37D0002B17D0019B19
:100B700018604360781CFFF7EFFE32000100280088
:100B8000FFF706FEFFF7E8FE0028CED02B692B62A8
:100B900000232B6103783A2B03D03060C5E7009027
:100BA000E8E70130FFF7D8FE320001002800FFF728
:100BB00031FFFFF7D1FE071EB7D0037801952C2B2C
:100BC000CED07D2B03D03060AFE7002300932023ED
:100BD000E360009B781CA36039E7002B00D120E77D
:100BE000A3E737601DE7C046A78B0010AC8B001051
:100BF000B28B0010FFFFFF7FF7B505000E000192DA
:100C00000F1E00D1144FFFF7B1FE002304003B601C
:100C100098420DD02800FFF79FFE3A000100200007
:100C2000FFF7F8FE051E05D12000FFF7C9FE0024DE
:100C30002000FEBD019B002B0AD0FFF78DFE03783C
:100C40000500002B04D02000FFF7BAFE3D60EEE760
:100C5000002EEDD03560EBE71C060208002210B52F
:100C60001100FFF7C9FF10BD802233B5450AFFB060
:100C70006D02040029009200684607F077FD012309
:100C80006A46E405E40D69462800135501F0CAF9E7
:100C90007FB036BD10B5183909180B780020012B2C
:100CA00002D00800FFF7E0FF10BD0000F0B58DB0E6
:100CB0001D0015AB1B780E0003930023170005A938
:100CC00006AA0593069300F048F9041E4BD12F4B5A
:100CD0003200009306993B000598FFF74DFC002871
:100CE00051DD0C22210009A807F049FD022008AAC5
:100CF00007A9FF300794089400F08EFF002802D067
:100D0000652464422FE02900079800F04BFE00287C
:100D1000F6D1033008AA07A9FF3000F07DFF0028B4
:100D2000EED11299079800F0DBFD041E1BD109A932
:100D3000300000F02AF9041E15D112990A9800F02B
:100D40002BFD041E0FD1039A29000B9800F03CF9EB
:100D5000041E05D1139B002B08D1149B002B0DD131
:100D60000998FFF72DFE20000DB0F0BD13990998EA
:100D700000F006FC0028F0D00400F1E7149909986F
:100D800000F0D4FCF8E71424BBE7C046005F2D0058
:100D9000F0B58BB01F0010AB059204CB04911B780B
:100DA00006920793002309AA08A90600089309934D
:100DB00000F0D3F8041E22D1099800F06BF804006B
:100DC00007F0AEFC051E20D0114B020000930999DC
:100DD00023000898FFF7D0FB002813DD079B2200B3
:100DE0000393069B01970293059B29000093300013
:100DF000049BFFF75BFF0400280007F09BFC20002A
:100E00000BB0F0BD14246442F6E764246442F6E7B4
:100E1000005F2D0010B5010004000B4807F080FDB5
:100E2000002398420DD02100084807F079FD0123E6
:100E3000002806D02100064807F072FD43424341D6
:100E40005B00180010BDC0468F8D0010988D0010FB
:100E5000A08D001010B5010004000B4807F060FDE4
:100E6000002398420DD02100084807F059FD0123C6
:100E7000002806D02100064807F052FD43424341B6
:100E80005B00180010BDC046758D00107E8D0010EF
:100E90008A8D00100323584380089843043070471C
:100EA000F8B50D0000281FD000291DD0C3680860C8
:100EB000202B1CD184680F4F002C01D12000F8BDDD
:100EC000266A002E06D031000B4807F029FD0028C5
:100ED00002D16C602468EFE73100380007F020FD94
:100EE0000028F7D1AC60F5E701204042E7E7022097
:100EF000FBE7C046AE8D0010A88D0010F0B50700CE
:100F00000D00002491B001AE002D02D1280011B0D7
:100F1000F0BD296A002904D0380007F001FD00283F
:100F2000F4D0AB68002B06D00E2C12D8A20095513D
:100F300001341D00E8E72B68002BFAD1002C0AD001
:100F4000013CA3009B591B68002BF2D1002CF7D168
:100F5000EFE70025DAE72500D8E7F8B50E002E21E7
:100F6000170007F0CFFC041E0CD0451C2E212800D2
:100F700007F0C8FC002805D0001B013838600020AD
:100F80003560F8BD16204042FBE770B50500002033
:100F90000C00FFF7FBFC2800FFF760FE002803D0E1
:100FA0002100FFF77DFF70BD05204042FBE70023D5
:100FB00004220133002901D1904203D952001D2B94
:100FC000F7D1023318007047F0B50C0087B001006C
:100FD000C1480592FFF792FF002800D18BE2836899
:100FE0000093019300231F0004930393019B002BA4
:100FF0006CD1009BDB680193202B00D07CE2009E2B
:101000003100B648FFF77AFF051E00D1E6E0037E07
:10101000059A9A4200D0E1E00100B148FFF76EFF67
:10102000002800D1D4E0836923702900AD48FFF780
:1010300065FF1423002800D0836963602900AA4853
:10104000FFF75CFF0123002802D0C3685A1E9341BA
:1010500023722900A548FFF751FF002800D1BAE00C
:101060008369E360002329006376A148FFF746FF08
:10107000002807D001699F4807F052FC002801D1E1
:10108000012363762300627E49331A70009E002F8D
:1010900000D031E231009148FFF730FF002800D145
:1010A000A1E02278037E9A4200D09CE03100924871
:1010B000FFF724FF002800D10AE130238269551E82
:1010C0006B43E3181A760223019393E001998B484E
:1010D000FFF714FF002802D08668002E03D1019B81
:1010E0001B68019382E731008548FFF707FF00285E
:1010F0004BD0002503690293824AAB0099580298AD
:1011000007F00EFC002800D1F9E10135042DF3D1E0
:1011100000257D4AAB009958029807F001FC071E94
:1011200005D00135172DF4D10527183D7F42310038
:101130007648FFF7E3FE002801D08369049331006D
:101140007348FFF7DBFE002804D0C1698069FFF710
:101150002EFF03906B1C18D0039B002B15DDA922DA
:101160006B00E31852009A5C012A04D12A0004990A
:101170000E32D20011515422FF329B5C012B04D15C
:101180000E35ED00039B65196B603668A5E7614974
:10119000029807F0C5FB0028F7D131005B48FFF744
:1011A000ADFE002806D0A2235B00E35C012B01D139
:1011B0008369A36631005648FFF7A0FE0028E4D0FB
:1011C0004623FF33E35C012BDFD18369E366DCE771
:1011D00001277F4229E7FA231B0142E73668002EE8
:1011E00000D00DE752E73668002E00D052E7012309
:1011F00035000193002E00D098E031004648FFF7FB
:101200007DFE002800D0FFE031004448FFF776FE65
:1012100000280ED00D236B43E3182A33FF331B78CD
:10122000012B06D1C2682F33511E8A416B43E3184C
:101230005A7031003A48FFF761FE00280ED00D23A6
:101240006B43E3182C33FF331B78012B06D1C268A4
:101250002F33511E8A416B43E3181A743100314811
:10126000FFF74CFE00280CD00D236B43E3182C3302
:10127000FF331B78012B04D12F336B438269E318B2
:101280009A7431002848FFF739FE002800D1CBE0DE
:10129000C368102B00D0C7E082680D2123200023F3
:1012A0006943684361180290002A00D1BCE01F0026
:1012B0003237FF37CF5D012F04D10298C7189069EC
:1012C0002C37C8550133032B00D1ADE01268EBE792
:1012D0000123050001938DE7758D0010578C0010D8
:1012E000D68B0010DD8B0010E58B0010F08B00100A
:1012F000FC8B0010098C00100E8C0010B78B0010B6
:10130000D08D0010E400020888000208C18B001094
:10131000C98B0010CE8B00101A8C0010B38D0010FA
:10132000318C0010398C0010488C00103100864838
:10133000FFF7E4FD002800D15FE78768002F00D1A8
:101340005BE739008148FFF7D9FD00282DD00369FC
:101350007F491800029307F0E3FA002827D13900EB
:101360007C48FFF7CBFD00280CD00D236B43E3181E
:101370002E33FF331B78012B04D12F336B4382694B
:10138000E318DA6139007448FFF7B8FD00280CD083
:101390000D236B43E3182F33FF331B78012B04D14C
:1013A0002F336B438269E3181A623F68C6E76B49C3
:1013B000029807F0B5FA0028F7D139006548FFF721
:1013C0009DFD00280CD00D236B43E3183033FF3311
:1013D0001B78012B04D12F336B438269E3185A62C7
:1013E00039005D48FFF78AFD0028DED00D236B43EE
:1013F000E3183033FF331B78012BD6D12F336B43E7
:101400008269E3189A62D0E70D236B43E3182D330A
:10141000FF331B78012B00D0F6E62F336B43826934
:10142000E318D2B25A61EFE631004D48FFF766FD8E
:1014300030236B43E31800284CD082699A70310046
:101440004848FFF75BFD002846D03022C169836918
:101450006A430B43591E8B41A2185374002D1CD1B3
:1014600031004148FFF74AFD1423002800D083696A
:10147000636331003D48FFF741FD22003832002808
:1014800030D0C368591E8B41137031003848FFF7C4
:1014900035FD002828D08369E363019B022B2AD104
:1014A000009E31003348FFF729FD00281FD08269D4
:1014B000D3B2022B1BD13027551E6F43E21913768E
:1014C00031002D48FFF71AFD002801D083693B55F4
:1014D0000123F9E59870B2E7302301226B43E3184A
:1014E0005A74BBE71070D0E7FA231B01D4E73668C3
:1014F000002ED6D1ECE70027380007B0F0BD1F4919
:10150000029807F00DFA002800D040E6310011489B
:10151000FFF7F4FC002806D0A1235B00E35C012B5D
:1015200001D18369236631000B48FFF7E7FC0028EF
:1015300000D12AE64423FF33E35C012B00D024E6EC
:101540008369636621E6C046B78B0010D08D00101A
:10155000248C0010C18B0010C98B0010298C001046
:10156000528C00105A8C0010DD8B0010E58B00109F
:10157000F08B00100E8C0010578C0010658C001042
:10158000F0B5554BBDB003AC63600E000B1DE360BE
:10159000524B0C36236101236662514E0A00A6624B
:1015A000CE1826634F4E083266630E001036E6638F
:1015B0004D4EA26126640E001436A6644B4E4C4A72
:1015C000E6640E00183666654A4E0025A6650E00D4
:1015D000E26102221C36039163612262E36263646A
:1015E0002365A560A563E3652666434EA36666662C
:1015F0000E002036E666414E626726670E002436EE
:10160000A6673F4E2392E6670E00283624963D4E8D
:10161000269325960E002C3627963B4E2993289626
:101620008E182A96394E32922B96CE1C2D96384E15
:101630002C952E960E0030363096364E2F953196DC
:101640000E003436339635920A0038323692324ADA
:10165000324E37923C31324A39910100314834964A
:1016600038933A923B93FFF749FC0600A84219D001
:101670008368AB4216D00C236B43E71831007868BF
:101680000193FFF73BFC002809D0C368042B06D167
:10169000BB68012B12D0002B07D0022B13D00135D1
:1016A000132DE8D100203DB0F0BD019BC169E25887
:1016B00083690B43591E8B411370F0E7019B8269CC
:1016C000E3581A60EBE7019B1749E2588369DB0195
:1016D0005B181360E3E7C046908C00109D8C0010EF
:1016E000B58C0010C28C0010CC8C0010D68C001071
:1016F000AA8C0010DE8C0010E58C0010F38C00101A
:10170000FD8C0010088D0010148D0010218D00102C
:101710002B8D0010388D00104D8D0010428D001063
:10172000598D0010668D001000003140F8B50E0094
:1017300001001648FFF7E2FB011E08D08368002B6A
:1017400005D01348FFF7DAFB0400002C01D100207C
:10175000F8BDA4680F4FA1683800FFF7CFFB350034
:101760000028F2D0C368042BEFD18369321D2B60AF
:10177000036824689B6921006B60D36F38000133D4
:10178000D367FFF7BBFB0835EAE7C046BB8D001007
:101790000F8E0010C78D001070B50C0001001648A8
:1017A000FFF7ACFB051E24D001001448FFF7A6FB91
:1017B000002806D0E378012B03D10069FFF72AFB4C
:1017C000207029000E48FFF799FB002806D02379E6
:1017D000012B03D10069FFF73DFB60702900094828
:1017E000FFF78CFB002804D06379012B01D18369BA
:1017F000A370002070BDC046768C0010798C00105C
:10180000848C00108C8C001070B504000D0086B024
:101810000021142201A806F0B2FF29002000FFF7E2
:101820006DFB0400002C18D021001C48FFF766FB5C
:101830000028F7D00569002D0AD0194E2900300084
:1018400007F06EF800280BD1310001A807F072F8FC
:10185000210001A8FFF752FB0400200006B070BD74
:10186000104E2900300007F05BF80028ECD029006A
:101870000D4807F055F80028E6D00C4E290030003E
:1018800007F04EF80028DFD02900094807F048F893
:101890000028DDD121000748C1E7C046D08D0010E7
:1018A000F88D0010E18D0010E88D0010F08D001013
:1018B000D58D0010DB8D001010B5FFF71FFB012444
:1018C000002809D08168002906D00448FFF716FBDC
:1018D000002801D0C468E4B2200010BD6D8D001056
:1018E000F7B5040000200D00FFF750F82000FFF7C7
:1018F000B5F9071E4AD001002648FFF7FFFA041E7B
:1019000006D1012676423800FFF75AF83000FEBDB6
:1019100001002148FFF778FF210006001E48FFF76D
:10192000CBFF0090002E2BD03069FFF773FA6B4687
:1019300000261B782870EB7021001848FFF764FF21
:10194000210000901548FFF7B7FF009B0190002B86
:1019500019D01869FFF77EFA6B461B7968702B71F6
:1019600021000F48FFF750FF210000900C48FFF7BF
:10197000A3FF009B002BC4D09B696871AB70C2E7CA
:1019800001267642D8E701267642E9E70526764227
:10199000BCE7C046768C0010798C0010848C001057
:1019A0008C8C0010F0B5050085B000200C00FEF70F
:1019B000EDFF2800FFF752F90190002800D115E152
:1019C00001008C48FFF79AFA051E00D10AE18A4F00
:1019D00001003800FFF718FF290006003800FFF764
:1019E0006BFF002E00D1E1E09422B3695200DBB21C
:1019F0002370A0542200303213703623FF33E0549A
:101A000000237E4F290038000093FFF7FDFE2900D8
:101A100006003800FFF750FF002E00D1C9E0F36840
:101A20005A1E93412A22DBB2FF326370A054220077
:101A3000313213709B235B00E054714F2900380052
:101A4000FFF7E2FE290006003800FFF735FF002E01
:101A500000D1B2E0F3685A1E93412C22DBB2FF3270
:101A60002374A0542200403213709C235B00E05486
:101A7000644F29003800FFF7C7FE29000600380030
:101A8000FFF71AFF002E00D19BE09622B3695200A7
:101A9000DBB26361A05463643A23FF33E0545A4ECF
:101AA00029003000FFF7B0FE290007003000FFF7E3
:101AB00003FF002F00D188E02200BB692C32DBB28B
:101AC00013703222FF32A05422005C3213709F2226
:101AD0005200A05422002D32137099225200A054BB
:101AE00022005D3213704022FF32A05422002E32B9
:101AF00013703422FF32A05422005E321370A023F0
:101B00005B00E05401994148FFF7F8F90600002F07
:101B100068D02E220123FF32A354D218A3543022BE
:101B2000FF32A354D218A35423000222384FFE33AD
:101B3000FF3201009A87DA873800FFF765FE31002F
:101B400005003800FFF7B8FE0390002D41D0AB69C7
:101B50000293304F31003800FFF756FE3100050088
:101B60003800FFF7A9FE002D38D0AD692200210012
:101B70002300533229317033FF32FF31029E5D6002
:101B80001E606E46367B08331670507002329942E2
:101B9000F4D1A12302225B00FF32E2520233E2526F
:101BA0000198FEF70DFF009805B0F0BD01235B42E0
:101BB00027E701235B4200933FE701235B42009349
:101BC00056E701235B42009369E701235B420093E0
:101BD00098E701235B4202950093BAE701235B4239
:101BE0000093C3E701235B420093D2E705235B42E6
:101BF0000093D8E7758D0010578C0010B38D00103E
:101C0000318C00101A8C0010488C0010B78B00101B
:101C1000C18B0010C98B0010DC23F0B59B0585B08B
:101C20000093002302AD019502901848184C0668F5
:101C30006B60306A0768002F07DBA34203D10120E5
:101C4000404205B0F0BD0133F4E7A342F7D06B4644
:101C5000C3600123BC3683603368C0180023066864
:101C6000002E03DAA342EAD00133F8E7A342E6D01C
:101C7000A02300981B06984201D00098E1E7029B40
:101C8000002013606B680B60DBE7C046F80A0208AF
:101C9000983A00000122F0B50024184B0668196834
:101CA00032400B6ABC310D6815495D191F68002F61
:101CB00006DB8C4202D101204042F0BD0134F5E741
:101CC0008C42F8D0002A00D106000120DE60986026
:101CD00000202C68002C03DA8842ECD00130F8E7B1
:101CE0008842E8D0DB68002A00D11B68A0220020CF
:101CF00012069342E1D01800DFE7C046F80A020856
:101D0000983A00000A4B37B51B780500013B0024C8
:101D1000012B05D8074B01A80193FFF7BBFF040077
:101D2000002D02D0280004F081FA20003EBDC046FC
:101D3000181002080101013A07B5034B01A80193ED
:101D4000FFF7A8FF0EBDC0460101003210B5FFF736
:101D5000F3FF002801D106F0F7FE10BDF8B506002C
:101D600008001700FFF7CEFF1D4B1B68002B20DA81
:101D700080241C4B1C4DA4002B511C4B1C481B6881
:101D80001A009832196812688A18116808401949AF
:101D9000014311601A00903212681B689B181022D0
:101DA00019681142FCD0012004F040FA2E51FFF7CF
:101DB000CDFF002F0CD005F063F9C02201230E499E
:101DC0005200885803438B5005F096F905F040F90E
:101DD000300005F087FA002004F0B6FDFBE7C046AE
:101DE000000126400040001600002040F80A0208CA
:101DF000FCFF00000300FA0500002640C02201237A
:101E0000044910B55200885803438B5005F074F90B
:101E100010BDC04600002640F8B5284B421E050004
:101E20009A4248D8264B1A78002A44D10124254FDB
:101E30001C703B78244E002B07D1FFF7DFFFE12217
:101E4000D200B358A343B3503C70C02201210024F8
:101E50005200B3588B43B3501C4B1D801C4BA20047
:101E600099184988A94221D8D35A9D4200D21D0011
:101E7000184B20001C7005F027F9C22328005B00D6
:101E8000F65806F09FFA144A144B05F01BFC05F0B7
:101E900039FB11231C1B103BA3408019C01A80B2D0
:101EA00005F000F9FFF7AAFF0020F8BD01340D2C62
:101EB000D5D1013CDCE701204042F6E76F17000076
:101EC0002406020825060208000026402206020811
:101ED0003C8F00102006020833DFC14F1C409F3F9B
:101EE000C0220120044952008B5883438B500022AA
:101EF000024B1A707047C0460000264024060208B4
:101F0000C0220120024952008B5883438B507047F6
:101F100000002640014B18607047C046F80A0208CE
:101F2000044B1B681A00BA3212881B6A5043C0184F
:101F30007047C046F80A02081D4B98420FD010D8CF
:101F400040282FD005D8002830D0102828D0194894
:101F50001EE0802828D080235B009842F7D11448E7
:101F600016E0154B984214D008D8A0231B069842BF
:101F70001CD0124B9842EAD1A0200BE0104B9842A3
:101F80000AD0104B984209D00F4B9842DFD10F482E
:101F90007047A420C003FBE70D48F9E70D48F7E7B9
:101FA0000D48F5E70D48F3E70D48F1E70020EFE7AE
:101FB00006005200FF005200010000F0090000A0DE
:101FC000040000F0050000F0030000F001005200E2
:101FD00002005200030052000100500002005000B5
:101FE0000500520010B50020FFF79AFF0A4B1C684D
:101FF0002300BC331B68C0180368002B0ADB074BA7
:102000001868FFF799FF012263689A609A68002AAE
:10201000FCD110BD0248FCE7F80A020828060208B5
:102020000200500070B5C40506000D00E40D20D17B
:1020300000291ED005F0F6F80F4B104A1A605C60BC
:102040009E60DD600E4B1B685233197800290BD05F
:1020500004F055F8FA21890005F07EF901000948DD
:1020600005F07AF9084BC1188020400006F064FDA5
:1020700070BD0648FCE7C0462806020800010005BE
:10208000F80A0208C0EA21014826000006005200B2
:102090000E4B10B51B689C695B69001BC0090001F1
:1020A000C0181F231A40032907D8C9008B408A4053
:1020B00004689C432243026010BD0439C9008B4070
:1020C0008A4044689C4322434260F5E7F80A0208CC
:1020D000F8B51F0006AB15001A7806000C00FFF7D4
:1020E000D7FF012211001740A140A7403368A40088
:1020F0008B433B433360074B1B6881331B78F618D7
:102100000F2319001D40A140A54032688A432A438D
:102110003260F8BDF80A0208064B1B68BC331B6826
:10212000C3181B68002B03DA89B241600020704796
:102130000148FCE7F80A020801008A000368002B46
:1021400004DA89B2C2608160002070470048FCE771
:1021500001008A00064B1B68BC331B68C3181B6850
:10216000002B03DAC36800200B6070470148FCE7CE
:10217000F80A020801008A00024B1A68002A00D1FE
:10218000186070473C060208F0B52C246043154CDB
:102190001F0024681D0A2018FF2425402740124CE8
:1021A0001B0C26680760346A45608360BA3636883F
:1021B00077433F1907612F0080376D017F01E719D1
:1021C00064190A4D47611F043B43641923600023CF
:1021D0008361059BC2610162002B01D01B88838152
:1021E000F0BDC0463C060208F80A020808100000CC
:1021F000F0B5836885B002AD2B80154B02681B6873
:10220000066A1B8F476A9B186B8043680095826A39
:10221000C16A040003930369C068FFF7B5FF00219A
:102220003B000A0000913000FFF7AEFF216B280051
:1022300003F0B2FF0022AB5E002B06DB1F2213402F
:102240001E3A9A401300034A136005B0F0BDC04621
:10225000F80A020800E100E0F7B52C25134C6843AA
:10226000266869433418256901937118002D19D027
:102270008869002818D12E68002E15DA67680124B5
:1022800026004B689E40B44613689EB263461B040A
:102290001E431660EA608C61BC40019BA4B24B6295
:1022A000AC60FEBD0248FCE70248FAE73C060208C3
:1022B00004028A0007028A0073B5002642690400FE
:1022C000D56801962B0CB34221D01B041360136810
:1022D000194B00691B68BC331B68C3181B68B342E9
:1022E00015DA01A9FFF736FFB0420CD10198E26977
:1022F00003681E0CDBB29A4205D9226A9B009B58E8
:10230000002B00D0984731002069FFF705FFADB2E0
:10231000002D09D063691D6000251B68636AAB420C
:1023200005D098476562A56163691B6873BDA36AA0
:10233000002BF8D09847F6E7F80A02082C2310B5CE
:102340004343034A1068C018FFF7B6FF10BDC046EC
:102350003C060208F8B5194B0F001B681A0033320F
:102360001278824227D9002925D01F250A681540F6
:1023700021D11900BA310C88114E60431C6AD20871
:10238000041929007868346006F0F9F92900200062
:10239000FFF7C2FE3A0029003068FFF7CFFE041EA7
:1023A00007D101003068FFF7B7FE03002000002BC3
:1023B00000D00448F8BD0448FCE7C046F80A02080B
:1023C0004006020801018A0003018A0010B5002AB4
:1023D0000DD1002914D10B4B1A681300BA331B8896
:1023E0005843136AC018084B1860080010BD002934
:1023F00006D0064B196019005A60FFF7ABFFF5E7EE
:102400000348F3E7F80A020840060208040000083F
:1024100003018A00F7B5184F04003B680191DE689C
:102420003368834226D90025A94202D1FEF755F828
:10243000050038680368002B1ADA1F2201232240A6
:10244000934064097268A4001419226813420DD0E5
:102450009A43226000240021FFF75EFE019B002BBF
:1024600002D12800FEF73DF82000FEBD034CF2E744
:10247000034CF3E7034CF7E740060208020188002B
:102480000301880004018A000A4B1B68DB681A6894
:1024900082420DD959681F23420918401E3B8340D0
:1024A000920050581840431E9841034BC018704783
:1024B0000248FCE7400602080001880004018A0087
:1024C00070B59621002003F01FFF0021080002F0E4
:1024D000F9FF444244412D4B64421C402C4B050003
:1024E0000020E41802F06CFF012002F04DFF0020F4
:1024F00002F076FE04F096FE264E33683F331B78DA
:10250000002B03D0012003F04FFB0500002D00D06D
:10251000214C33683F331B78012B03D9022003F091
:1025200043FB0500002D00D01C4C0021012003F0CE
:1025300099F9002800D01A4C002002F0B9FF051EBE
:102540000ED103F0B7F91223FF33984208D10121CD
:10255000280002F08FFF002800D00D4C04F062FE2E
:1025600003F00AFA002800D00E4C0021080003F006
:1025700079F9002800D00C4C0021080002F07AFF05
:10258000002800D0024C200070BDC046F1F0E5FEEE
:102590000F0F1A01F80A02082F0F1A012E0F1A0145
:1025A0004E0F1A013F0F1A014F0F1A0130B5134C8D
:1025B000C000031908300019002901D0072A06D9E4
:1025C00001220021524219605A6006C030BD0C4CF5
:1025D0002468A5696469491BC909090109191960B9
:1025E000043101601F21032A03D8D20091405960B1
:1025F000ECE7043AD20091404160E7E7FC0A0208A8
:10260000F80A0208F0B5C400454E002900D17AE06E
:10261000072A00D977E0002336199D00DF004D1905
:102620000133F551152BF8D1143B93403D497360AC
:1026300009194B603C49032509194B603B49384F48
:1026400009194B603A4909194B603A4909194B601D
:10265000394909194B60394909194B6038490C1936
:1026600051000E00374963600C68B540210080318D
:1026700009789200023189080918C900C9194D600A
:102680000F25210095408131097802318908091808
:10269000C900C9194D6035001035AC4621006646A9
:1026A000032582310978B540023189080918C9002B
:1026B000C9194B602100833109782B430231890805
:1026C0000918C900C9194B60FE2301219B008434FD
:1026D0001A402378012502339B081818531CC000A8
:1026E0009940C71901200B00911C88409540032692
:1026F00003431D43D31C9E402E43072505329540BE
:102700002E437E60F0BD0023012118003419494298
:10271000E050E21808335160A82BF9D1F2E7C04627
:10272000FC0A0208040B02080C0B0208140B020836
:102730001C0B0208240B02082C0B0208340B0208A5
:102740003C0B0208F80A0208C14BF0B51B6887B0C1
:102750001A00BA321188186A8A001218D0680290DA
:102760000088059002984088009002988768C068A9
:1027700004900598013808280AD804F0E3FD6700A2
:10278000270046005E09C000FF00E70276008400D3
:10279000B04C6A46029B928A85211A806A46802044
:1027A00012885C605A80049A9F60DA60A84B4901E5
:1027B0001B6840031A6ABA33505018885158800079
:1027C00080180021FFF7A8FC07B0F0BD009AA24BCB
:1027D000D20099184968049C0C4001D001F030F9EE
:1027E000481C01D101F02FF90098922801D901F07D
:1027F0002DF9D258002A01D101F02BF91368394381
:102800000B4004990B431360C3E7009A924BD1002D
:102810005A185268501C01D101F01EF900989228F4
:1028200001D901F01CF9C958002901D101F01AF9A8
:102830000B68174205D018007840024201D001F021
:1028400014F913403B430B600024A2E7009B922B3A
:1028500001D901F00DF9DA007F4BD358002B01D1DB
:1028600001F009F91F68002493E7022F01D001F05D
:1028700005F9049C794B143C604244417848644219
:102880000440E41885E7002F01D101F0FAF8049B19
:10289000052B01D901F0F8F8724B1B681A78002A51
:1028A00025D09A683A60DA687A606F4ABA605A78D6
:1028B000002A1ED01A6AFA609A6A3A616B4A7A61F3
:1028C0005A6ABA61DA6AFA61694A3A629C78002CFB
:1028D00012D01A6B00247A629A6BBA62654AFA6265
:1028E0005A6BDB6B3A637B63634BBB6351E73A60C4
:1028F000DDE7FA60BA61E9E77C623C6349E7002FF3
:1029000001D101F0C4F85D4CF0223900200005F03F
:102910002DFF03F0C1FC002810D0FFF7D1FD2000EF
:1029200001F062FC564B04001A78002A00D030E710
:10293000002800D02DE701321A702AE7504B1B788F
:10294000002BECD1E378002BE7D0E379002BE4D027
:10295000230055331D7803F08DFC0028DDD102F0F3
:1029600053FE002805D102F043FE280002F06CFE61
:10297000D3E702F053FE0028F5D0CEE7009B672B8B
:1029800000D18BE018D82F2B00D1C6E107D82C2B13
:1029900000D192E02D2B00D1EBE02E4CF9E6009B0C
:1029A000322B00D1B2E1662B34D0302BF5D1380078
:1029B00002F010FE0024ECE6009B6E2B00D13BE100
:1029C00008D86C2B00D133E16D2BE6D104F06CF903
:1029D0000024DEE6009B702B00D13FE100D233E102
:1029E000712BDAD13B78002B01D001F05CF8254A3D
:1029F0000425101DC06F01268446397A634500D036
:102A000065E1002004F0BCF8441EA04144421E4889
:102A10000440BEE61D4B5A68002F10D11C491140DE
:102A20001B220A435A6059681A4A1143596059686F
:102A30001143596059680A435A600024A9E6E82105
:102A4000154889010240114359605A680240F3E772
:102A5000F80A0208FF0F1A01FC0A0208F90F1A010E
:102A600007F0E5FE3C0702082000890035008B00D6
:102A70004A008D005F008F00740091004806020834
:102A800038070208940F0208FE0F1A0100002640C2
:102A90000000FC0F003A0280FF00FC0F03234B43B1
:102AA0009B181A68002AFCDA80220024D968520593
:102AB0000A43DA605C605B686BE60024B125994BE1
:102AC000ED001C80984B1C80984B1B683F331B7893
:102AD0009C4201D900245CE6002C1ED102F03AFF92
:102AE000002818D0200002F0E5FE022836D1002C84
:102AF00017D18F4A8F485359184080239B0518439C
:102B000050510021200002F0ADFE0123A340854A70
:102B100011880B4313800134D6E7200003F030F80E
:102B2000DEE70326824AA30083499B185A58120FF6
:102B3000324204D05A58120F3240012A06D10122E3
:102B4000A2401000784E3288104330805A5879489D
:102B500010408022920510435850D2E7002CDAD161
:102B6000734A744953590B40802189050B435351D3
:102B7000D1E76C4B1B88002B0FD102F0EBFE041E3B
:102B800000D106E66D4C40E0013D02F081FD0228D7
:102B900005D0002DF8D16A4CFBE5684DF5E7002D16
:102BA000F9D00026664C09E0013D02F0DBFE00286A
:102BB00001D000F0B1FF002DF6D101365B4B1B6850
:102BC0003F331B789E4200D9E3E50123B3409BB21B
:102BD0000193544B019A1B881342EED0022130001E
:102BE00002F040FE002EE0D0300002F0D3FF0028BB
:102BF00001D000F0A0FF002DDFD0013DF4E7C020A0
:102C0000800501439950D8E7013C02F0ABFE002853
:102C100002D1002CF8D1BEE7002CBCD0B122C023D9
:102C20004349D20088589B0503438B500024B0E5EC
:102C300003F0E8FF0024ACE53800431E9841C0B221
:102C400004F042F80024A4E53878072801D900F000
:102C500021FF797804F008F800249AE53B78002BEE
:102C600001D000F01AFF7968CAB20F2A01D900F02A
:102C700017FF0125334C8D40A446201D3A7AC66FBC
:102C8000B34208D1002003F041FF441EA04144425A
:102C90002D4804407DE5D800604404682C4214D0DF
:102CA000022A08D0032A0BD0002AEBD14368DB07A5
:102CB000E8D4254C6DE543681342E3D1224C68E526
:102CC00043685B07DED4204C63E50133D8E7022973
:102CD0000BD0032910D0002916D11A4CD8000019A6
:102CE0004068304210D1184C53E5D8008018406835
:102CF000084209D1144C4CE5124CD8000019406828
:102D0000284201D100F0D2FE013377E63A893888B3
:102D1000796803F039F804003BE5380003F0EAF87D
:102D2000040036E54406020846060208F80A0208CE
:102D300000002640FFFFFFCFFC05000040420F00CF
:102D4000FA0F1A01940F0208FE0F1A01B44A127802
:102D5000002A01D100F0ADFE00980838632801D99F
:102D600000F0AAFE04F0EEFAD100DD00F10013013C
:102D700021012F0140014E01A80660016E017C0176
:102D80009401D4011402BC02590372038B03A403FF
:102D9000B803CC03DA03E803FC0310041E042C047C
:102DA00045045404620470059905C305F4054906F9
:102DB000A806A8066206A806A806A806A806A806E9
:102DC000A806A806A806A806A806A806A806A80693
:102DD000A806A806A806A806A806A806A806A80683
:102DE000A806A806A806A806A806A806A806A80673
:102DF000A806A806A806A806A806A806A806A80663
:102E0000A806A806A806A806A806A806A806A80652
:102E1000A806A806A806A806A806A806A806A80642
:102E2000A806A806A806A80664008400A400BA00A4
:102E300001227C4D6B78E91C01932B792E7803934A
:102E4000FBB22A706A70CB77002B0ED12A71280052
:102E500001F0CAF9041E00D19BE46B461B792E7069
:102E60006B706B461B7B2B7193E400232B71EEE799
:102E7000012100226B4D6B78281D01932B792E7850
:102E80000393FBB229706A70C377022B0ED12971AC
:102E9000280001F0A9F9041E00D17AE46B461B79E1
:102EA0002E706B706B461B7B2B7172E42A71EFE7FF
:102EB0005C4D2B786E1D0193F37F28000393012353
:102EC0002B70F37701F090F9041E00D161E46B469A
:102ED0001B792B706B461B7BF3775AE4514D2B7893
:102EE0006E1D0193F37F2800039301232B700023B1
:102EF000F37701F079F9041E00D14AE46B461B799F
:102F00002B706B461B7BF37743E40023454D280071
:102F10006E796B7101F068F9041E00D139E46E71AD
:102F200037E4404D6B7A280001930023AE6E6B723C
:102F3000AB6601F059F9041E01D1FFF72AFC6B467C
:102F40001B79AE666B72FFF724FC002F01D100F0F5
:102F5000B6FD3F331B78BB4201D200F0B3FD002326
:102F6000304D012F0DD1AE7AAB72280001F03CF943
:102F7000041E01D1FFF70DFC012F05D1AE72FFF742
:102F800008FCEE7AEB72F0E7EE72FFF702FC012329
:102F9000244D2800EE79EB7101F026F9041E01D1D1
:102FA000FFF7F7FBEE71FFF7F4FB00231D4D280040
:102FB000EE79EB7101F018F9041E01D1FFF7E9FB7E
:102FC000EE71FFF7E6FB3B0016485A1E93410500E1
:102FD00055352E782B7001F007F9041E01D1FFF74B
:102FE000D8FB2E70FFF7D5FB01230E48451CEE7F62
:102FF000EB7701F0F9F8041E01D1FFF7CAFBEE7779
:10300000FFF7C7FB00230748451CEE7FEB7701F075
:10301000EBF8041E01D1FFF7BCFBEE77FFF7B9FB1D
:1030200038070208480602080123C94D28002E7AF5
:103030002B7201F0D9F8041E01D1FFF7AAFB2E7202
:10304000FFF7A7FB0023C24D28002E7A2B7201F058
:10305000CBF8041E01D1FFF79CFB2E72FFF799FB02
:10306000BB48FBB20500013B5A4253410024563590
:103070002E782B70037AA34201D1FFF78AFB01F06F
:10308000B3F8041E01D1FFF784FB2E70FFF781FB1C
:10309000052F01D900F019FD3800AD4D012304F0D2
:1030A00047F90316191C1F226E7D6B75280001F06D
:1030B0009BF8041E01D1FFF76CFB052F01D9FFF728
:1030C00068FB380004F034F91215181B1E21AE7D80
:1030D000AB75EBE7EE7DEB75E8E72E7E2B76E5E74B
:1030E0006E7E6B76E2E7AE7EAB76DFE76E75FFF75E
:1030F00050FBAE75FFF74DFBEE75FFF74AFB2E76E2
:10310000FFF747FB6E76FFF744FBAE76FFF741FB18
:10311000052F01D900F0DCFC380000238C4D04F0B1
:1031200007F90316191C1F226E7D6B75280001F02C
:103130005BF8041E01D1FFF72CFB052F01D9FFF727
:1031400028FB380004F0F4F81215181B1E21AE7D80
:10315000AB75EBE7EE7DEB75E8E72E7E2B76E5E7CA
:103160006E7E6B76E2E7AE7EAB76DFE76E75FFF7DD
:1031700010FBAE75FFF70DFBEE75FFF70AFB2E7621
:10318000FFF707FB6E76FFF704FBAE76FFF701FB58
:103190003868052801D900F09EFC6D4C3B7922006F
:1031A00004F0C6F8032E3C4A58662600A532A8361D
:1031B00015781370326818000192627DA63403926C
:1031C00002F060FF23786349D84004F0C5F8039B00
:1031D00030601C1E01D1FFF7DCFA5D4E300001F0BB
:1031E00003F8041E01D1FFF7D4FA3868052801D985
:1031F000FFF7CFFA330004F09BF84950575E656C37
:103200002600AC32B036157813703268180001927F
:10321000A27DAD34039202F035FFD3E72600B4322D
:10322000B83615781370326818000192E27DB53413
:10323000039202F027FFC5E72600BC32C03615789E
:103240001370326818000192227EBD34039202F09E
:1032500019FFB7E72600C432C836157813703268F4
:1032600018000192627EC534039202F00BFFA9E7B9
:103270002600CC32D03615781370326818000192CF
:10328000A27ECD34039202F0FDFE9BE7A5331D70B4
:10329000019BA8363360FFF77CFAAC331D70019BAD
:1032A000B0363360FFF775FAB4331D70019BB83642
:1032B0003360FFF76EFABC331D70019BC03633607C
:1032C000FFF767FAC4331D70019BC8363360FFF700
:1032D00060FACC331D70019BD0363360FFF759FA8A
:1032E0003868052801D900F0F9FB194B3A791C0020
:1032F00004F01EF803323D48535E1D00A634A83585
:10330000267822702A6801925A7DA5330392187894
:1033100002F0B8FE23780F49D84004F01DF8039B53
:1033200028601C1E01D1FFF734FA094D280000F077
:103330005BFF041E01D1FFF72CFA3868052801D97C
:10334000FFF727FA2B0003F0F3FF3E454C535A6179
:103350004806020840420F001D00AD34B035267803
:1033600022702A6801929A7DAC330392CFE71D0048
:10337000B534B835267822702A680192DA7DB433E4
:103380000392C4E71D00BD34C035267822702A6838
:1033900001921A7EBC330392B9E71D00C534C835CB
:1033A000267822702A6801925A7EC4330392AEE7CF
:1033B0001D00CD34D035267822702A6801929A7E7D
:1033C000CC330392A3E7A6331E70019BA8352B6074
:1033D000FFF7DFF9AD331E70019BB0352B60FFF7AF
:1033E000D8F9B5331E70019BB8352B60FFF7D1F9C2
:1033F000BD331E70019BC0352B60FFF7CAF9C53382
:103400001E70019BC8352B60FFF7C3F9CD331E70CA
:10341000019BD0352B60FFF7BCF9D84D2E00AB7C5B
:10342000A236019333782800039301233770AB74DD
:1034300000F0DAFE041E01D1FFF7ABF96B461B7BEF
:1034400033706B461B79AB74FFF7A3F9CB4D2E009D
:10345000A336337828000193EB7C37700393012364
:10346000EB7400F0C1FE041E01D1FFF792F96B4628
:103470001B7933706B461B7BEB74FFF78AF9BF4DEA
:103480002E002B7FD6360193337828000393012337
:1034900037702B7700F0A8FE041E01D1FFF779F9F1
:1034A0006B461B7B33706B461B792B77FFF771F9EB
:1034B000B24800240500D8352E882F80837FA34290
:1034C00001D1FFF766F900F08FFE041E01D1FFF76E
:1034D00060F92E80FFF75DF9A84800240500DA3571
:1034E0002E782F70837FA34201D1FFF752F900F0AD
:1034F0007BFE041E01D1FFF74CF92E70FFF749F94E
:1035000001239E4D2800AE7FAB7700F06DFE041EB8
:1035100001D1FFF73EF9AE77FFF73BF90023974D56
:103520002800AE7FAB7700F05FFE041E01D1FFF7ED
:1035300030F9AE77FFF72DF9904800240500D43517
:103540002E782F70C37EA34201D1FFF722F900F03D
:103550004BFE041E01D1FFF71CF92E70FFF719F97D
:10356000864800240500D5352E782F70C37EA342EF
:1035700001D1FFF70EF900F037FE041E01D1FFF76D
:1035800008F92E70FFF705F901237C4D2800EE7E27
:10359000EB7600F029FE041E01D1FFF7FAF8EE7673
:1035A000FFF7F7F80023754D2800EE7EEB7600F06C
:1035B0001BFE041E01D1FFF7ECF8EE76FFF7E9F8E9
:1035C0006E4D2E006B7FD73601933378280003931E
:1035D000012337706B7700F007FE041E01D1FFF75F
:1035E000D8F86B461B7B33706B461B796B77FFF704
:1035F000D0F8624B5C79002C00D072E23A689A6293
:103600007A68DA62BA681A63FA685A63FFF7C1F82F
:1036100001235A4D28006E796B7100F0E5FD041E00
:1036200001D1FFF7B6F86E71FFF7B3F838680528D7
:1036300000D959E2514B03F07BFE031B222930379E
:103640001A00012196321E7B15881973B98818005B
:10365000118000F0C9FD041E38682CD1052801D95D
:10366000FFF797F8454D03F063FE4D6A8DADC3D962
:103670001A00012198325E7B15885973E6E71A001B
:1036800001219A329E7B15889973DFE71A00012188
:103690009C32DE7B1588D973D8E71A0001219E324F
:1036A0001E7C15881974D1E71A000121A0325E7CB6
:1036B00015885974CAE7052800D918E22F4B03F082
:1036C00037FE03080D12171C1E7396331D80FFF77B
:1036D00060F85E7398331D80FFF75BF89E739A3332
:1036E0001D80FFF756F8DE739C331D80FFF751F8FD
:1036F0001E749E331D80FFF74CF85E74A0331D804E
:10370000FFF747F86B7A002B03D0280000F0B8FCD5
:10371000A8662B00A5331878002801D0FFF739F8E8
:1037200002F0B0FC2B00A6331B781549A835994050
:103730004B08181803F010FE2860FFF72AF8AB7A40
:10374000002B05D02900012000F0B8FC2B1DD86704
:103750002B00A5331878012801D0FFF71AF802F0E2
:1037600091FC2B00A6331B780549A83599404B08DE
:10377000181803F0F1FD2860FFF70BF8480602085F
:1037800040420F00EB7A002B06D02900022000F007
:1037900095FC2B008C3318602B00A5331878022879
:1037A00001D0FEF7F6FF02F06DFC2B00A6331B786C
:1037B000EB49A83599404B08181803F0CDFD286057
:1037C000FEF7E7FF2B00A5331878032801D0FEF79A
:1037D000E0FF02F057FC2B00A6331B78E049A83528
:1037E00099404B08181803F0B7FD2860FEF7D1FF89
:1037F0002B00A5331878042801D0FEF7CAFF02F089
:1038000041FC2B00A6331B78D549A83599404B08BD
:10381000181803F0A1FD2860FEF7BBFF2B00A533AD
:103820001878052801D0FEF7B4FF02F02BFC2B001E
:10383000A6331B78CA49A83599404B08181803F0DD
:103840008BFD2860FEF7A5FF3A68C64B0024DA66B8
:103850001A00B988703211801A00B9797232117069
:103860001A00F979733211701A0039897432118093
:103870001A00B97A763211701A00F97A773211701B
:103880001A00B989783211801A00B97B7A32117026
:103890003A8A7C331A80FEF77CFFB24D6E7A002E96
:1038A00000D027E1012328006B7200F0E9FBA86635
:1038B000280000F099FC041E03D0AE666E72FEF77D
:1038C00068FF2B00A5331B78002B01D0FEF761FFAA
:1038D00002F0D8FB2B00A6331B78A149A8359940EC
:1038E0004B08181803F038FD2860FEF752FF3A68BD
:1038F000002A00D101E13F331B789A4200D9FFE052
:103900007B681E785D789C78D8781979954B012A68
:1039100010D11A00843216701A00853215701A0000
:10392000863214701A0087321070883319700024A0
:10393000FEF72FFF1A00903216701A0091321570A0
:103940001A00923214701A00933210709433EDE71B
:10395000012F06D1834A927A002A09D0824CFEF7C1
:1039600018FF022F04D17F4AD27A002A00D0CAE081
:103970003F331B78BB4200D2C8E0002F00D1C8E023
:10398000784D2900012F12D1380000F097FB2B1D34
:10399000D867AF72280000F027FC041E16D0002361
:1039A000012F0DD12A1DD367AB72FEF7F2FE022064
:1039B00000F084FB2B008C3318600123EB72E9E7E5
:1039C0002A008C321360EB72FEF7E3FE2B00A53366
:1039D0001878431E012B01D9FEF7DBFE02F052FBE3
:1039E0002B00A6331B785E49A83599404B08181860
:1039F00003F0B2FC2860FEF7CCFE5A4D2E002B7D62
:103A0000A4360193337828000393012337702B7574
:103A100000F0EAFB041E01D1FEF7BBFE6B461B7BE8
:103A200033706B461B792B75FEF7B3FE01224D4BAD
:103A300000249A719F64FEF7ACFE0024FEF7A9FEF5
:103A40004A4CFEF7A6FE494CFEF7A3FE474CFEF794
:103A5000A0FE464CFEF79DFE444CFEF79AFE434CFA
:103A6000FEF797FE414CFEF794FE404CFEF791FEA8
:103A70003E4CFEF78EFE3D4CFEF78BFE3C4CFEF7B7
:103A800088FE3C4CFEF785FE3A4CFEF782FE394C30
:103A9000FEF77FFE374CFEF77CFE364CFEF779FED4
:103AA000344CFEF776FE334CFEF773FE314CFEF7D6
:103AB00070FE2E4CFEF76DFE2C4CFEF76AFE2E4C6F
:103AC000FEF767FE2C4CFEF764FE284CFEF761FE05
:103AD000264CFEF75EFE254CFEF75BFE234CFEF700
:103AE00058FE264CFEF755FE204CFEF752FE1F4CAA
:103AF000FEF74FFE224CFEF74CFE1F4CFEF749FE30
:103B00001D4CFEF746FE184CFEF743FE164CFEF722
:103B100040FE154CFEF73DFE002D01D1FFF74DF89C
:103B2000B122C0201749D2008B58800503438B5027
:103B30000024FFF742F8002D01D1FFF73EF8124BA9
:103B400010491C88019B114A1C40B3005B1899580E
:103B5000002C01D1FFF753F80D4801409950E7E7D9
:103B600040420F00480602082D0F1A01FF0F1A01EC
:103B7000F90F1A01FE0F1A01BD0F1A01590F1A0190
:103B80003E0F1A010000264046060208FC05000010
:103B9000FFFFFFCF73B593220020354BD100354C8A
:103BA000591A0919013A0860002AF7D132491960F7
:103BB0003249996032491961324999613249196231
:103BC0003249996232491963324999633249196419
:103BD00032490968080040300078042800D9304A8A
:103BE0009A640022052800D92E4A1A654A680124E1
:103BF0001000083098652C48644218662B48DC6732
:103C000058662B4898662B4818672B4812189A67F5
:103C1000002215009818060008328036843035607E
:103C20000460802AF6D18522244B52010433DD67DB
:103C30000B6A68469B18802252039A6004236A46E6
:103C400013800B8F1E4905335380019502F0A4FAAF
:103C5000002800D001BE6B4600229B5E002B06DBD5
:103C60001F2213401E3A9A401300164A136073BD78
:103C7000FC0A02089C0400000800264000072640B9
:103C800004072640080726401007264084032640E4
:103C9000880326408C03264090032640F80A020839
:103CA00094032640980326400400264000FF03F0BA
:103CB000480526404405264060F00000940F0208A5
:103CC0004927001000E100E010B5244C2368002BC8
:103CD00043D01A78002A0AD0DA6899682020FEF7C3
:103CE00091FC23688920DA689968FEF75FFC2368F5
:103CF0005A78002A16D09A6A196A3520FEF782FC93
:103D000023684A20DA6A596AFEF77CFC23688B2014
:103D10009A6A196AFEF74AFC23688D20DA6A596AA2
:103D2000FEF744FC23689A78002A16D09A6B196B28
:103D30005F20FEF767FC23687420DA6B596BFEF78F
:103D400061FC23688F209A6B196BFEF72FFC2368A8
:103D50009120DA6B596BFEF729FC10BD3C07020875
:103D6000022817D006D8002827D0012810D002201A
:103D700040420CE01223FF3398420DD01423FF334E
:103D800098420CD0033B9842F1D1FA20C001704711
:103D9000886CFCE7886AFAE780200002F7E7084BA6
:103DA0001B68413318780138431E9841054B404247
:103DB000184080231B02C018E9E70348E7E7C04624
:103DC000F80A0208FE7FFFFF00127A0002235B421E
:103DD00010B51360314B14001B681A003E32127884
:103DE000824258D9052856D803F0A2FA03192E4367
:103DF000494F0B7B002B4ED04B7A002B08D00B0089
:103E00007A331B78022B03D08B6E2360002010BD09
:103E10000B0096331888FFF7A3FF2060F6E74A7B74
:103E2000002A38D03F331B78002B0AD08B7A002B26
:103E300007D00B0088331B78022B02D00431CB6FE4
:103E4000E3E70B009833E5E78A7B002A23D03F3372
:103E50001B78012B0AD9CB7A002B07D00B009433A7
:103E60001B78022B02D08C310B68CEE70B009A3303
:103E7000D0E7CB7B002B0ED00B009C33CAE70B7C2A
:103E8000002B08D00B009E33C4E74B7C002B02D0E4
:103E90000B00A033BEE70248B9E7C046F80A0208A3
:103EA000FE0F1A01194B00B513600023052809D82D
:103EB00003F03EFA030A13191F250023087B9631ED
:103EC000984206D1180000BD0023487B98319842E3
:103ED000F8D00B8800211160F4E70023887B9A3129
:103EE0009842F6D1EEE70023C87B9C319842F0D18E
:103EF000E8E70023087C9E319842EAD1E2E70023FC
:103F0000487C9842DED0A031E3E7C046FE0F1A019C
:103F1000032819D004D801280FD028D948790DE0FA
:103F20001223FF33984214D01423FF33984212D047
:103F3000033B98420BD00F4805E088794342584133
:103F40000C4B4042184070470231C87FF6E7C879F1
:103F5000F4E7087AF2E70131CB7F002BEBD0064B78
:103F60001B68413318780138431E9841E8E7002068
:103F7000E9E7C046FE0F1A01F80A020810B51B4B0C
:103F80001B683E331B7883422DD905282BD803F0BC
:103F9000CFF9030C12181E240B7B002B23D00B002F
:103FA00096331888FFF7B4FF10BD4B7B002B1AD057
:103FB0000B009833F5E78B7B002B14D00B009A3362
:103FC000EFE7CB7B002B0ED00B009C33E9E70B7C9B
:103FD000002B08D00B009E33E3E74B7C002B02D074
:103FE0000B00A033DDE70248DEE7C046F80A02080E
:103FF000FE0F1A010300A8331B6810B50400002B44
:1040000002D00848584310BD0300A533187802F0C9
:1040100039F802000120A63423789840400880181F
:10402000D840F0E740420F0010B5040001F0E4FD75
:10403000002801D0044810BD0449200001F052FEC0
:104040000028F8D0F6E7C046FD0F1A01102700003F
:1040500070B50400150001F00DFA002801D00748E2
:1040600070BD2900200001F02DFA0028F7D12000B2
:1040700001F0B8F90028F3D0F1E7C046FD0F1A01AE
:10408000030010B50400963318882100FFF768FE7E
:10409000030000209A1C0FD0220070321188814248
:1040A0000AD0E06E7334584303F056F921784B1E62
:1040B0009941013103F050F910BD000070B50025A1
:1040C0000C00A84221D01B4B1B683F331B78834256
:1040D0001BD301281BD10B0098331888FFF740FE33
:1040E00023002200843385321B78117886342578AA
:1040F000821C1BD000291BD0002D06D0584303F092
:104100002BF9290003F028F90500280070BD0228CA
:10411000FBD10B009A331888FFF722FE2300220000
:10412000903391321B7811789234E0E70025ECE768
:104130000D00EAE7F80A0208F8B504000F000129AB
:1041400032D10300817A427B04309833C66F8330CA
:104150001B8805780020814225D0824231D018008A
:104160002100FFF7FDFD184BC018184B984228D8C6
:104170006B1E9D41164B6D421D40164BED18237969
:10418000002B1AD0AE421CD3134B9E4219D82100EB
:104190003800FFF793FF301A464270410F4E4042FD
:1041A0000F4B3040C018F8BD0300C17A827B9A33B0
:1041B0008C301B880668C579CCE7AE4201D3094B29
:1041C000E3E70748EFE7C04600F7C2FF0087930325
:1041D000C863E3FF20BCBE0080F0FA0202F0E5FEF7
:1041E000FE0F1A0180D1F008F0B504008BB0002852
:1041F00001D100F092FF0700404EA53733683878B0
:104200003E331B78984207D300203D4B0593059D14
:10421000002D06D03B4D6EE005AA2100FFF742FEBF
:10422000F5E7022820D01223FF33984245D0012819
:1042300000D071E0344B1B68002B13D01A78002A91
:1042400010D05A68A16C8A420CD19A68E16C8A42FB
:1042500008D1DB68226D934204D1230054331B78CC
:10426000102B59D0294D46E0274B1B68002B22D03C
:104270005A78002A1FD01A69A16A8A421BD15A694A
:10428000E16A8A4217D19A69216B8A4213D1DA69AD
:10429000616B8A420FD11A6AA16B8A420BD15A6AAA
:1042A000E16B8A4207D19A6A216C8A4203D1DB6AA8
:1042B000626C934230D0164D1DE0134B1B68002BEF
:1042C00018D09A78002A15D022005632D978127860
:1042D00091420FD11A6BA16D8A420BD15A6BE16DDD
:1042E0008A4207D19A6B216E8A4203D1DB6B626EE0
:1042F000934211D0074D28000BB0F0BDF80A020818
:10430000FE0F1A019F0F1A013C070208570F1A01EE
:10431000580F1A01560F1A0101F0BAF902281DD0E0
:104320006379002B1AD0D74AA36A9B18D64A9342C6
:1043300001D900F0F5FEE36A013B632B01D900F0DF
:10434000EFFE236BD14A013B934201D900F0E8FE16
:10435000636B013B934201D900F0E2FEA379002B8D
:104360000ED02279A36C002A00D120E2C84A9342E1
:1043700001D900F0D8FEE36C002B01D100F0D3FE90
:10438000237B002B0ED033683E331B78002B09D0E3
:104390002300963318882100FFF7BAFD002801D0CA
:1043A00000F0C4FE637B002B0ED033683E331B78D5
:1043B000012B09D92300983318882100FFF7A8FDA5
:1043C000002801D000F0B5FEA37B002B0ED033688F
:1043D0003E331B78022B09D923009A331888210019
:1043E000FFF796FD002801D000F0A6FEE37B002B2E
:1043F0000ED033683E331B78032B09D923009C333E
:1044000018882100FFF784FD002801D000F097FEF6
:10441000237C002B0ED033683E331B78042B09D944
:1044200023009E3318882100FFF772FD002801D079
:1044300000F088FE637C002B0ED033683E331B787F
:10444000052B09D92300A03318882100FFF760FD50
:10445000002801D000F079FE01F07CFA00285DD13F
:10446000637A002B5AD0237B002B01D100F070FE21
:104470002300963318882100FFF772FC854BC01883
:10448000854B984201D900F063FE844AA36E9B18C5
:104490002279002A00D18CE1814A934201D900F0AF
:1044A00057FEE36E7F4A013B934201D900F050FE74
:1044B000230070331B887C4A013B9BB2934201D995
:1044C00000F046FE230072331B78042B01D900F064
:1044D0003FFE23007433754A1B88934201D900F0D4
:1044E00037FE230076331B780F2B01D900F030FE06
:1044F000230077331B780F2B01D900F029FE23000E
:1045000078336B491B888B4201D900F021FE2300D0
:104510007C331B88934201D900F01AFE33683F3385
:104520001B78002B13D0A37A002B10D0012001F0B0
:1045300027FB00280BD133683F331B78002B05D0B5
:1045400001212000FFF7F8FD002800D0594D336805
:104550003F331B78012B00D83BE1E37A002B00D1DD
:1045600037E1002D00D0C6E6022001F009FB00284B
:1045700000D120E1237F002B00D02EE1637D002BB2
:1045800000D147E63368029340331B78002B00D1FB
:1045900040E63D7821002800FFF7F0FC002800D01D
:1045A00038E6029B3E331B789D4200D232E1424BFB
:1045B0000493049B002B00D02CE605AA3878210038
:1045C000FFF704FC3D4B059A050004909A4200D881
:1045D00020E6002800D01DE62300A8331B68002B2E
:1045E00000D117E62200A6321178354A354F5343E1
:1045F0000292BB4200D90DE6032900D90AE6A37D49
:10460000002B1DD0336840331B78012B18D92300B1
:10461000AC3318782100FFF7B1FC002801D000F07E
:104620006EFC2300AD331A7803331B6802994B43A9
:10463000BB4201D900F063FC032A01D900F05FFC02
:10464000E37D002B40D0336840331B78022B3BD9ED
:104650002300B43318782100FFF790FC002801D024
:1046600000F077FC2300B5331A7803331B680299F6
:104670004B43BB4201D900F06CFC032A01D900F086
:1046800068FC21E000DC0BFFC0EA2101E703000029
:1046900080F0FA0218FCFFFF18DDF50500CA91FE54
:1046A00080BA8C01FEFF0300FE1F0000FF01000026
:1046B000FF1F0000BF0F1A01FE0F1A013F0D03007C
:1046C00040420F0080D1F008237E002B1DD03368BC
:1046D00040331B78032B18D92300BC3318782100F2
:1046E000FFF74CFC002801D000F02BFC2300BD3369
:1046F0001A7803331B6802994B43BB4201D900F07F
:1047000020FC032A01D900F01CFC637E002B1DD085
:10471000336840331B78042B18D92300C43318782E
:104720002100FFF72BFC002801D000F027FC23001C
:10473000C5331A7803331B6802994B43BB4201D936
:1047400000F01CFC032A01D900F018FCA37E002B0A
:104750001DD0336840331B78052B18D92300CC3388
:1047600018782100FFF70AFC002801D000F047FC70
:104770002300CD331A7803331B6802995943B94299
:1047800001D900F03CFC032A01D900F038FCE37E9B
:10479000002B52D1637F002B6FD1A37C002B00D064
:1047A00091E0E37C002B00D0A0E09B4DA3E59B4A69
:1047B000DDE59B4A71E633683F331B78012B06D950
:1047C00002212000FFF7B8FC002800D1D2E6954D69
:1047D00091E5002D00D1CDE68DE52300D6331B7881
:1047E000012B0AD0002B03D0032B08D08E4D82E57D
:1047F000E379002B00D0C1E6F8E7237AF9E7631CE0
:10480000DB7F002BF2D0336841331B78012B00D1C2
:10481000B4E6EBE704AA21002800FFF743FB882356
:104820005B00984200D1F5E41423FF33984200D195
:10483000F0E4032800D0BCE6ECE42300D4331E7877
:1048400021003000FFF79AFB002814D12300D53354
:1048500002931B78042B0ED805AA21003000FFF725
:10486000B5FA002807D1029B059A1B78DA4013009D
:104870006E4A93428ED96E4D3DE52300D7331B78A7
:10488000002B03D0012B05D06A4D34E5237A002B91
:1048900083D1F9E7237F002BF6D02300D6331B7892
:1048A000012BF3D0002B0CD0032BEDD1631CDB7F4D
:1048B000002BE9D0604B1B6841331B78012BE3D1FF
:1048C0006BE7E379E3E7637D002B01D15B4D12E5F4
:1048D0002000FFF78FFB2300A2331978013102F08B
:1048E0003BFD524B984200D85BE7EFE7637D002B1E
:1048F00000D15AE72000FFF77DFBB84200D954E70A
:104900002300A33302931978013102F025FD2379A6
:10491000002B0BD04A4B984200D946E7A37F002BCF
:1049200006D1237D002B39D1464DE4E43B4BF2E721
:1049300023000222D8331B88FF32934204D022D8AE
:10494000002B28D0012B24D1617D002921D0022603
:10495000934208D03C4AB619934204D03B4A0436ED
:10496000934200D0073E2000FFF744FB2300DA33D8
:104970001978013102F0F0FC310002F0EDFC2B4B14
:104980009842CED905E030498B42DDD02F498B4289
:10499000DAD02F4DAFE401262E48E7E7E37C002B69
:1049A000C2D02000FFF726FBB84200D9FDE6270061
:1049B000E31C0393029BA4371978261D013102F0F2
:1049C000CBFC3978013102F0C7FC144B9842ABD8CC
:1049D0009621002001F098FC2378002B49D06378C1
:1049E000002B10D0E31CD87F012806D9631DDB7F84
:1049F000002B33D102F0D2F932E002F029FA00287C
:104A0000F4D0154D77E4F07F022801D00528EDD1D0
:104A100002F07CFAF3E7C0468C0F1A0100E1F505BD
:104A200000AB8704BE0F1A01AF0F1A010084D7171D
:104A30008F0F1A018E0F1A01F80A02088D0F1A0142
:104A400040787D018B0F1A01010200000103000074
:104A5000890F1A0100127A006F0F1A0102F070F923
:104A60000028CED102F0E6FAA378002B74D002F031
:104A7000BFFABC4B1B6841331B78012B09D100F0F6
:104A800093FD631CDB7F002869D0002B01D100F06F
:104A900095FD0822B44B1E68237A164066D0002B81
:104AA00004D17B2001F0DCFB00F050FD237F002BC4
:104AB0000ED02300D6331E7800F05CFC864207D06F
:104AC00002F0D2FA002800D045E3300000F044FCA8
:104AD00000F0DEFD6379022870D1002B01D100F0D7
:104AE000CBFDA379002B0ED0E06C002808D023006A
:104AF00054331B7808220093216D0023FDF7E8FA58
:104B0000A06C00F0AFFDA37C002B04D02300A233E7
:104B1000187800F055FCE37C002B03D0029B18783A
:104B200000F032FC237D002B02D0387800F058FBD7
:104B30002600122796363388FF37BB427CD12300EC
:104B4000A5331978002977D1012000F08BFE0028C9
:104B50005ED0864DFFF7CFFB02F05AFA89E7002BB3
:104B600097D002F05FFB00F009FD92E7002B9DD08B
:104B700002F058FBA06D00280FD0E36D002B0CD085
:104B800033003200216E0096FDF7A2FA0096330042
:104B90003200616EE06DFDF79BFA23005633187802
:104BA000002800D0012000F0D9FC714800F0B0FCD2
:104BB000002800D17AE76F4DFFF79DFB002B90D0C6
:104BC00002F030FBA06B002810D0E36B002B0DD05F
:104BD0000026216C330032000096FDF779FA00962A
:104BE00033003200616CE06BFDF772FA636B226B8D
:104BF000E16AA06A00F05AFD002802D05E4DFFF77E
:104C00007AFB5E4800F0F0FD002800D169E7F5E787
:104C1000012100F02FFC00280BD1237B002B14D0A6
:104C20003188002000F01EFE00280ED0544DFFF702
:104C300062FB544DFFF75FFB230098331988012076
:104C400000F010FE0028E8D083E7A37B002B0AD0F9
:104C500023009A331988022000F004FE002802D0B5
:104C6000494DFFF748FBE37B002B3ED1237C002B13
:104C70004CD1637C002B5AD100F06CFE637A002883
:104C800066D1002B00D18BE002F0CCFAE36E05A8D0
:104C90000593230070331B888380230072331B78B5
:104CA0008371230073331B78C371230074331B8813
:104CB0000381230076331B788372230077331B78BC
:104CC000C372230078331B88838123007A331B78D7
:104CD000837323007C331B88038200F06BFE002863
:104CE0003CD12A4800F0F0FE36E01E4B1B683E33F4
:104CF0001B78032BBAD923009C331988032000F0BA
:104D0000B1FD0028B2D0224DFFF7F5FA154B1B6814
:104D10003E331B78042BACD923009E331988042022
:104D200000F0A0FD0028A4D01A4DFFF7E4FA0D4BC7
:104D30001B683E331B78052B9ED92300A0331988AE
:104D4000052000F08FFD002896D0134DFFF7D3FA11
:104D5000002B25D100F010FE002821D00F4DFFF7C9
:104D6000CAFAC046F80A0208000027404E0F1A018E
:104D700040420F005A0F1A015F0F1A01B80B0000D2
:104D80004F0F1A010F0F1A014D0F1A01400D0300AA
:104D90004C0F1A014B0F1A014A0F1A013F0F1A014B
:104DA0002300A53302931978002000F063FB00284C
:104DB00000D03EE72300A633197800F083FB0028DB
:104DC00000D036E73388BB4217D0C34F3B683F3330
:104DD0001B78002B75D0012000F0D2FEA37A0028AA
:104DE0001CD0002B38D102F01DFA012000F0DCFEAF
:104DF000002831D0B94DFFF77EFA029B1B78002BBB
:104E0000E3D1637B002B00D1A3E6230098331988FC
:104E1000012000F027FD0028D7D09AE6002B1BD0F8
:104E2000230084331B7805AE3370230085331B7851
:104E30007370230086331B78B370230087331B788D
:104E4000F370230088331B78337102F0EBF93100E3
:104E50000120FFF7E9F8CBE73B683F331B78012BD4
:104E60002FD9022000F08CFEE37A00280BD0002B13
:104E700027D102F0D7F9022000F096FE002820D0BA
:104E8000974DFFF738FA002B1BD0230090331B7887
:104E900005AE3370230091331B7873702300923377
:104EA0001B78B370230093331B78F3702300943383
:104EB0001B78337102F0B6F931000220FFF7B4F825
:104EC000DCE7012000F0A8FAA37D00281AD0002B0F
:104ED00010D0022000F0A0FAE37D00281DD1002BA5
:104EE0001DD02300B5331A78013B19780220FFF753
:104EF000AFF82CE0012000F0A1FA0028E9D0794DAC
:104F0000FFF7F9F9002BE4D02300AD331A78013B09
:104F100019780120FFF79CF8EFE7002B14D03B68CD
:104F200040331B78032B17D9032000F075FA237E3A
:104F3000002826D0002B0FD1032000F07FFA002894
:104F40000AD0694DFFF7D7F9022000F077FA002860
:104F5000E5D0664DFFF7CFF93B6840331B78042B53
:104F60001AD9042000F058FA637E00282FD0002BB5
:104F700012D1042000F062FA00280DD05C4DFFF73A
:104F8000BAF9002BE8D02300BD331A78013B197819
:104F90000320FFF75DF8D2E73B6840331B78052B11
:104FA00020D800F0C3F9A37F002836D1002B38D0D9
:104FB0002300D8331F889E7800F0C2F9380000F033
:104FC00085F9300000F096F900F0A4F929E0002BF3
:104FD000E2D02300C5331A78013B19780420FFF78B
:104FE00037F8C9E7052000F017FAA37E002809D09A
:104FF000002BD6D1052000F021FA0028D1D03D4D5C
:10500000FFF779F9002BCCD02300CD331A78013B80
:1050100019780520FFF71CF8EFE7002B01D100F00D
:105020008FF900F02DF9E37E002819D0002B01D173
:1050300000F030F9637F002B04D02300D7331878B9
:1050400000F034F923002C4F55331E783B78B342DF
:105050001BD002F009F8002813D0284DFFF74BF9B8
:10506000002BE7D02300D4331F785E7800F012F9CC
:10507000380000F0D5F8300000F0E4F800F0F4F863
:10508000D8E7300000F0E0FA3E7000F0BDFAE379B6
:10509000002835D0002B0ED1A32001F0E1F800F05C
:1050A000B3FA002807D001F0DFFF0028D5D100F0C7
:1050B000B5FA0028D1D12378002B08D0637D002BCE
:1050C00005D02300A8332079196801F01DF902F0FA
:1050D000A9F8FFF710F9C046F80A02082F0F1A01C5
:1050E0002E0F1A019E0F1A019C0F1A019D0F1A0113
:1050F0009B0F1A019A0F1A01400702085C0F1A0150
:10510000002BD8D000F080FA0028D4D101F0ACFFF9
:105110000028A2D100F06CFACDE7104DFFF7EBF8B4
:105120000F4DFFF7E8F80F4DFFF7E5F80E4DFFF7CD
:10513000E2F80E4DFFF7DFF80D4DFFF7DCF80D4DEF
:10514000FFF7D9F80C4DFFF7D6F80C4DFFF7D3F861
:105150000B4DFFF7D0F80B4DFFF7CDF8FE0F1A01FE
:10516000EF0F1A01EE0F1A01DF0F1A01DE0F1A01FD
:10517000DD0F1A01DC0F1A01DB0F1A01DA0F1A0119
:10518000CF0F1A011F0F1A0170477047F0230A044E
:105190001B0330B51A400F240B0023401A43084B61
:1051A0001D68830228691B188020C0011A501858F6
:1051B0002040401A411E884102494042084030BD0B
:1051C000F80A02080300C200044B10301B6880027A
:1051D0001B69C0580F2318407047C046F80A0208E0
:1051E000064B00021B68190088311A680B680449D5
:1051F000D21813680B40184310607047F80A020871
:10520000FF00FFFF054B1B681A0088321B681268FD
:105210009B181868000AC0B27047C046F80A020816
:1052200010B5A022F0240549D200240100028B58B9
:105230002040034C23401843885010BD00002640F6
:10524000FFF0FFFF10B5A022E0240549D200E401E1
:1052500000038B582040034C23401843885010BD56
:1052600000002640FF8FFFFFA02280230349D200C9
:1052700088581B0203438B507047C04600002640ED
:10528000A023034ADB00D0580004C00F7047C0467B
:1052900000002640A0220349D2008B580248034058
:1052A0008B50704700002640FF7FFFFFC021054A5A
:1052B000890000021368084003490B40184310603E
:1052C0007047C04600002740FFFCFFFF0549064A23
:1052D00010B58B58054C2340054C2040184388508E
:1052E00010BDC0460000264004050000FEFCFFFF84
:1052F000010300000449054A10B58B58044C000412
:1053000023401843885010BD0000264004050000CB
:10531000FFFF00FF80230349034A1B06885803430D
:105320008B5070470000264004050000024A034BE2
:10533000D058C00F7047C04600002640040500004A
:105340000349044A8B585B005B088B507047C0468A
:105350000000264004050000A02210B503240449E3
:10536000D2008B582040A3431843885010BDC0463C
:1053700000002640A023034ADB00D0580323184036
:105380007047C04600002640064B00061B68190007
:1053900088311A680B68D21813681B021B0A18435D
:1053A00010607047F80A0208044B1B681A00883224
:1053B0001B6812689B181868000E7047F80A0208EC
:1053C000064B00021B6819008C311A680B680449EF
:1053D000D21813680B40184310607047F80A02088F
:1053E000FF00FFFF094B1B6840331B7883420BD93A
:1053F000074BE0228000C0188023920081581B06D2
:105400000B438350002070470248FCE7F80A02086B
:105410000000264001004A00064A030012680020EE
:10542000403212789A4204D9E033034A9B009858DC
:10543000C00F7047F80A020800002640002810D06C
:10544000094B1B6840331B7883420AD9E022074B83
:105450008000C018920083585B005B0883500020D6
:1054600070470348FCE7C046F80A020800002640DF
:1054700001004A0010B50B4B1B6840331B78834278
:105480000DD90F290BD8E0220F24074B8000C0183C
:1054900092008358A34319438150002010BD034854
:1054A000FCE7C046F80A02080000264001004A0056
:1054B000034BE0308000C0580F2318407047C046AF
:1054C0000000264010B50B4B1B6840331B7883420D
:1054D0000ED903290CD8E0223024074B8000C018D5
:1054E000920083580901A34319438150002010BD45
:1054F0000248FCE7F80A02080000264001004A00C2
:10550000024B18694007C00F7047C0460000274093
:10551000082310B504000B4A11680B431360FFF712
:10552000EFFF002808D1002C01D1074810BD012051
:1055300000F096FE013CF2E760426041024C4042BE
:105540002040F3E70000274002004A000821024AF9
:1055500013688B4313607047000027408021054A81
:10556000490200041368084003490B4018431060C7
:105570007047C04600002740FFFFFEFF802370B544
:10558000074D084C1B062A59012013432B5100F0EC
:105590004DFEC0232A59DB0513432B5170BDC04675
:1055A000000026403C050000024A034BD058800012
:1055B000C00F7047000026403C0500000349044A24
:1055C0008B58DB00DB088B507047C046000026403C
:1055D0003C0500000449054A80058B58800D9B0A54
:1055E0009B02184388507047000026403C0500008D
:1055F00080230349034A1B06885803438B50704796
:10560000000026400C050000024A034BD058C00F92
:105610007047C046000026400C050000C023074A22
:105620005B00D058803BFF3B184005D104495358DC
:105630005B005B08535070470248FCE700002640BF
:105640000C05000003004A0010B501240349044A78
:105650008B58A3431843885010BDC0460000264015
:105660000C050000024B984201D8024B18607047AD
:1056700000E1F5054C0702080349044A8B585B001A
:105680005B088B507047C046000026402C05000088
:10569000A6220549D2008B580220DB439B0702D08B
:1056A000012388581840704700002640F0B51600C6
:1056B0001F003B4A3B4B0C00D15885B00290019231
:1056C0000393002967DB3849384A4318934264D86A
:1056D000631E632B61D8364A731E93425DD8354AE8
:1056E0007B1E934259D8FA21F5308900FF3001F032
:1056F00033FE05003048310047437008381801F088
:105700002BFE802284461023002012020100114348
:105710000F004F43BC4500D30800013B5208002B4B
:10572000F4D12900254B614358434B08C01801F0C0
:1057300013FE234B984230D96D43224B2249E8187F
:1057400001F00AFE644360436421323001F004FE3C
:105750001E49704301F000FE03281ED8012801D81D
:10576000012358401A4A019B1A499B5800031940CB
:10577000194B0B431843019B03999850019B039AC3
:1057800000209A5802231343019A5350134B029A54
:105790001A6005B0F0BD1248FBE71248F9E7C046B1
:1057A000000026402C05000000DC0BFFC0EA2101B0
:1057B000E7030000CF07000080841E00B36D0200E5
:1057C000890200005DF70000BBEE0100A0BB0D00E8
:1057D00020FF000008C0FFFFF70300005007020889
:1057E00003004A0001004A00F8B5144C144D0700AC
:1057F0006359002B1FDB8023060062591B061343ED
:105800006351FFF745FF02280AD0002E03D1300074
:10581000002F0FD009E0012000F022FD013EF0E74B
:10582000381E07D00020864204D1635905485B002A
:105830005B086351F8BD0448FCE7C0460000264001
:105840002C05000002004A0003004A0010B5FFF7D3
:105850001FFF0023022801D1014B1B68180010BD57
:1058600050070208104B1B683E331B78834219D93E
:10587000042910D94B1EFF3B132B13D81F231940AB
:105880000A4B8000C018C02304229B00C150403343
:10589000C250002070470723D0301940034B8000CE
:1058A000C150F6E70248F5E7F80A02080000264072
:1058B00001004A00094A83009B18D02292009858A0
:1058C00007221040042807D1C022920098581F23B5
:1058D00003408020400018437047C0460000264027
:1058E00010B5FFF7E7FF02281CD005D8002824D008
:1058F000012814D0002014E01223FF33984214D062
:105900001423FF33984215D0033B9842F2D10C4A3E
:105910000C4BD358002BEDDA8020000201E00A4B3B
:10592000186810BDFFF792FFFBE7FFF7E9FD0028BD
:10593000E0D0F1E7024A054BEBE70548F1E7C04646
:10594000000026400C0500004C0702083C05000042
:1059500000127A00B023024ADB00D058C00F704713
:1059600000002640B223034ADB00D0580123184030
:105970007047C04600002640B1200B4BC0001A58AB
:105980000A491140802292050A43B0211A50C900E9
:105990005A580020520052085A5005495A5852008D
:1059A00052085A507047C04600002640FFFFFFCF04
:1059B0008C05000070B5B024224AE4001359002B76
:1059C0003DDBC17903684D1EA9419B0309069B0B72
:1059D0000B431351038984881B491B04E4040B40C7
:1059E000E40C2343194C1A4D1351FF24C37AE026CB
:1059F0001B0123408489F60024022C400F252343F9
:105A0000847A2C40C0252343847BAD0524072C4099
:105A10002343B124E400135183790E4C1B02155922
:105A200033400D4E35402B431351038A00201B0495
:105A300015590B40094929400B43135170BD0848C3
:105A4000FCE7C046000026400000FF01840500007E
:105A500000FF1F008C050000FFF8FFFFFFFF00FEA6
:105A600003004A00B023154ADB00D35810B5990350
:105A7000DB01DB0F890BC371114B0160D3580F247D
:105A8000D904DB01DB0D0381B123DB00D358C90C42
:105A9000818019002140817219092140C172D90207
:105AA0009B009B0F8373074BC90CD35881815A0508
:105AB000DB01520FDB0D8271038210BD0000264016
:105AC000840500008C050000F8B580230600050061
:105AD0000427264C264A1B06A1580B43A350B22389
:105AE000DB00E3583B4201D1002D1FD1B121C90099
:105AF0006358204A1A4080239B0513436350002EAD
:105B000001D0002D06D0B0228023D200A1581B0660
:105B10000B43A350FFF726FF002811D1002D0AD117
:105B2000002E11D0FFF728FF1348F8BD012000F028
:105B300097FB013DD3E7012000F092FB013DE9E72F
:105B4000002E01D0002DEDD0B122C0230020D200C4
:105B5000A1589B050B43A3508642E6D0681E8541A1
:105B60006842064D044B2840C018DEE7000026407E
:105B70008C050000FFFFFFCF02004A00FEFFB5FFCB
:105B80008030034BFF308000C058C00F7047C046C4
:105B9000000026409030034BFF308000C0580123A6
:105BA000184070470000264070B50E4B1B683F330D
:105BB0001A78431E9A4213D90B4B0C4D8000C4181F
:105BC00063590B4A01201A4080239B0513436351FC
:105BD00000F046FB002063595B005B08635170BD19
:105BE0000448FCE7F80A020800002640FC05000013
:105BF000FFFFFFCF01004A00F0B5204B1B683F3389
:105C00001B78834233D31E4B80001E4CC0180359AF
:105C1000002B2ADB8E78B31E0E2B28D84F787B1EE4
:105C2000112B24D80B78CD789C46002D21D1152B33
:105C30001DD970239C451AD80A79022A0AD07F23DD
:105C4000614619400B003F023B4336043343ED06E7
:105C50002B430351C0211207890503590A400A4901
:105C60000B401A4302510020F0BD0848FCE70848E9
:105C7000FAE7122BFBD93823DCE7C046F80A020802
:105C800000002640FC050000FFFFFFCF03004A0094
:105C900001004A0010B5104B421E1B683F331B78B1
:105CA000934216D97F221F248030FF300B4B800097
:105CB000C3581A400A701A0C2240180A8A701A0136
:105CC0002040E240487000209B009B0FCA700B717F
:105CD00010BD0348FCE7C046F80A02080000264051
:105CE00001004A00F8B5214B0F001B683F331A78BA
:105CF000431E9A4237D91E4B8000C41880230E00E1
:105D00001C4D1B0662591343635101221A4BE35881
:105D1000134218D1002E11D1002F18D06359174A01
:105D200001201A4080239B051343635100F098FA29
:105D3000635913485B005B08635113E0012000F0D6
:105D40008FFA013EE1E7002F01D0002EE6D0635923
:105D500000209B009B0F022B04D1C02362599B059E
:105D600013436351F8BD0748FCE7C046F80A020830
:105D700000002640FC0500003C060000FFFFFFCFAE
:105D800002004A0001004A00F7B5484B0091150097
:105D9000984200D987E09A4200D984E0444B994266
:105DA00000D980E00122434B1A70FF2845D80F2309
:105DB00007261C001840FF2D58D8FF222D01154042
:105DC0002843F025E0222C43F025D20232432D0354
:105DD0002B43394D07262F683D00BA352D886E4379
:105DE000350001963E6AAD192E68002EFCDA334D5F
:105DF0002E78334D002E03D0324EAE59002E50DA9D
:105E0000314E32493160324E32493160A321C900EE
:105E10006E58A6430643304C6E50285998430243AF
:105E200000202A512D4B009A1A60264BEA503B6AFB
:105E3000019AD31800225A60FEBD294B984205D81A
:105E40000F231840060000242000B4E7254B060A63
:105E5000984204D8FF2304011C402643F3E7F023B3
:105E600000021B01184006431F4BECE71C4A9542F9
:105E700005D82A04F0252D032A403243A8E72A0A30
:105E800012043243174EB54207D8F0262D053604CA
:105E900035402A43FF252D049AE72D062A43134D4A
:105EA00096E71348C3E71248C6E7C0460F0600004E
:105EB000FFFFFF0048070208F80A0208540702081B
:105EC000000026401C050000080126401F1F00009E
:105ED000040126403D3D000014050000440702086F
:105EE000FF040000FF0500000F0F000000000F0F6F
:105EF00001004A00F8B5144B984219D90027134BFA
:105F0000C018F6213F23124D124CF6302E5949008D
:105F10001E4001F021FA321A002F00D032183F2122
:105F20002B590A408B4313432B51002F09D0F8BD46
:105F3000094B984204D8EE33FF33181A0127E0E7E3
:105F400000204042F3E7C046EC8100000080FFFFE4
:105F50000000264018FF0000137E0000F0B589B055
:105F600003AC14220021200002F009FC2000FFF7FE
:105F700079FDB0231A4ADB00D25800239A4203DA93
:105F8000A37B023B5A1E9341E57900266A1E954188
:105F90000135B34221D0A488B4421ED0039B300007
:105FA0000193FFF79DFC2A00330007003100200019
:105FB00001F07EFA0C0005003300019A3100380030
:105FC00001F076FAE6076A083243630880185941FF
:105FD0002A00230001F04CFA0600300009B0F0BDA1
:105FE00000002640F0B50026244B85B01B68070052
:105FF0003F331B78B3423ED0B0423CD083423AD3C9
:106000000522310002A802F0BAFB02A93800FFF70E
:1060100041FE3B008033FF33194A9B009B58B3423B
:1060200029DA02AB1B79022B25D002AB5C78B44293
:1060300021D09D78B5421ED01B7838000193FFF720
:106040004FFC2A00330007003100200001F030FA35
:106050000C0005003300019A3100380001F028FAE5
:10606000E6076A0832436308801859412A00230072
:1060700001F0FEF90600300005B0F0BDF80A020894
:106080000000264010B5041E04D1FFF767FF00286A
:1060900006D008E0064B1B683F331B78834203D2CF
:1060A0002000FFF71DFC10BDFFF79CFFEFE7C04687
:1060B000F80A0208E02210B50124094B8000920082
:1060C000C018835880589B069B0F9C400F23184094
:1060D000FFF7D8FF63081818210001F03DF910BD43
:1060E0000000264010B50020FFF7E4FF0400FFF792
:1060F0005BF9411C4808001901F02EF910BD10B5DC
:10610000FFF7F0FF0400FFF77DF8411C4808001975
:1061100001F022F910BD0000144B30B51A680724B5
:1061200013002C331B781F2B15D883081D00A543A3
:106130002C1E0FD103342040A040814012689B00E8
:106140002032D3180A00FF2181401C6862401140B0
:106150006140196030BD802320401B061843802316
:106160009B011268C91889008850F3E7F80A0208F1
:10617000064B9A680300064810339B00824202D106
:10618000985899507047034AD058FBE700ED00E05B
:106190000000020800040010F8B506000D000028F9
:1061A0003AD00023C05E002828DB7188FFF7B4FFD7
:1061B0000024FF22032794460023F05E716883B217
:1061C0001F40FF006646BA4089013140D243B940C2
:1061D000002815DB114E83089B009B19C026B600D2
:1061E0009F593A40114399510D4B9A680D4B9A4271
:1061F00002D12900FFF7BCFF2000F8BD0A4CD8E708
:106200000F263340083B064E9B089B009B19DE6916
:1062100032401143D961E7E7034CEDE700E100E0CC
:1062200000ED00E0000002080100560070B5802576
:1062300004002D02AC4205D8064B18686043FAF7FB
:1062400043F970BD044B1868FAF73EF9034BE418A4
:10625000F0E7C04604010208000102080080FFFFC9
:1062600010B5034B1B785843FAF72EF910BDC04602
:10627000080102088022054B12069A64986C044BB0
:10628000C043C0171840034BC01870470000274098
:10629000FDFFB9FF0300460080220C4B1201985805
:1062A0005A68D2B2002A02D08022D2021043084A91
:1062B000995889B2002902D08021490208439B588D
:1062C0001B0C02D080239B0218437047000026401D
:1062D00004080000FEE7000002680A4B10B51A60CF
:1062E00042685A6082689A60C268DA6002691A611C
:1062F00042695A6182699A61C269DA61FFF7EAFF0D
:1063000010BDC046E0050208F0B51922002800D1F2
:106310004B322A4B8A4292411B6852421C00AC34D9
:1063200024881D68671903253E68AE4316433E6006
:106330001E68A4192768224E374027601C00AE341F
:1063400024881E68A7193E68AE4332433A601A6833
:106350001B4EA21814682640166000280ED000209C
:10636000102904D9213088428041404201300F2257
:106370005B681968914308431860F0BD1A005532F4
:1063800012788A42F3D21A005632127801208A42D9
:10639000EDD21A005732127800188A42E7D21A005A
:1063A0005832127828008A42E1D21A005932107805
:1063B0008842804140420430D9E7C046F80A0208CA
:1063C000FFFCFFFFB0235B055A782120002A01D093
:1063D0005878C0B27047B0235B059A89002A02D072
:1063E000988980B2704780204000FBE770B5FFF7C6
:1063F000F2FF8023194A5B00984215D111680F24DF
:106400000B0002229C3318680B6818180368A3431A
:10641000134303600800A0300B6801685B1819681B
:10642000A1430A431A6070BDB02412680C4B1100DE
:106430006405E3580B4D9C312B40C025106809685A
:10644000AD0041180868284003430B601100A031DB
:1064500013680A689B18044AA258E3E7F80A02087E
:1064600048180000FFFCFFFF4418000070B5FFF75C
:10647000B2FF8023154A5B0098420DD1136814497E
:106480001A009C3212681B689B181A6811408022FF
:10649000D2010A431A6070BDB02412680D4B11007E
:1064A0006405E3580C4D9C312B40C02510680968E9
:1064B000AD0041180868284003430B601100A0316B
:1064C00013680A689B18054AA258E3E7F80A02080D
:1064D000FF8FFFFF50180000FFFCFFFF4C1800006B
:1064E00010B5FFF778FF8023124A5B0098420DD168
:1064F000136811491A009C3212681B689B181A68AD
:106500001140C022D2010A431A6010BDB0211268A6
:106510000A4B4905CB58110009489C310340C02063
:106520000968126880005218116801400B4313601B
:10653000EBE7C046F80A0208FF8FFFFF1C180000B7
:10654000FFFCFFFF70B5FFF746FF80231A4A5B0090
:10655000984215D111680F240B0003229C33186850
:106560000B6818180368A343134303600800A030A6
:106570000B6801685B181968A1430A431A6070BD73
:10658000B02412680D4B11006405E3580C4D9C318A
:106590002B40C02510680968AD00411808682840E4
:1065A00003430B601100A03113680A689B18C122D5
:1065B0005201A258E2E7C046F80A02082418000077
:1065C000FFFCFFFFF8B51E4FC0253B682D011A00E8
:1065D0009C321B6812689B181E68FFF7FCFE340093
:1065E00080232C405B0098420ED10020FEF7ECFD8A
:1065F0000400FFF7E7FE01221300222801D86342BE
:10660000634113401800F8BD3B680E4F19009C31E0
:106610001A68086812181068384010601A6808680C
:10662000121828001768B043384310601B680A68C6
:106630009B1818682840001B431E9841C0B2E2E72F
:10664000F80A0208FFF3FFFF7FB5274B86000D0015
:10665000F458042901D0012927D100200FE0A368B4
:106660002B420BD1E36829001A685B680292019300
:10667000039302A8236898471C4B1C606469002C94
:106680000BD01B4B9842EAD1012DE8D1174B18488B
:106690001A68184B9A5104B070BD012DFBD1144BF0
:1066A0009842F3D0134B9C51F5E7022906D10F4BCA
:1066B0001B68181EEFD01C6903E01C006369002BE7
:1066C000FBD10020002CE6D0A3682B4209D1E3685F
:1066D00029001A685B6802920193039302A8236859
:1066E00098472469EEE7C046980702089407020815
:1066F000FF0042008007020870B50400FFF762FE49
:1067000085B2FFF768FE06000020FEF75DFD8023DE
:106710005B00002811D19E4211D1222D0FD8802577
:106720001E4B6D041B68240659681D4B2C40CA582B
:106730001C4D2A401443CC5070BD9E4228D0174AAD
:106740001268156A9E420ED162426241FF23524294
:106750009A43154BD21801212800FBF7EFFC0028C3
:1067600008D01248E8E762426241012352429A434C
:106770000F4BEFE7094B1B68BC331B68EB181A681B
:10678000002AFCDBEB6800201B0EA02BE9D1D3E72D
:10679000222DE6D9014B1B681D6AD5E7F80A0208CD
:1067A00018F00000FFFFFFFE01010030040042006E
:1067B0000300000C70B50500FFF704FF002834D07B
:1067C000F9F78BFE0600022D17D10120FFF794FF89
:1067D000041E0DD1FFF70AFE072215494B699343AA
:1067E0002A4013434B61022D15D1FFF779FE002497
:1067F0003000F9F776FE200070BD07220C493420E6
:106800004B6993431A00032313434B61FFF728FDA1
:10681000FFF72CFEE0E79120FFF722FDFFF792FE45
:106820000020FFF769FF0400E2E7024CE3E7C046FF
:1068300000002640030042001A4B1B6819008831F3
:106840001A68096851180968016219008C310968D1
:106850005218126842621A0046321278002A1FD07B
:106860009A68E0321268D2061AD5F222DB68D201A9
:106870009A580260F022D2019A5842600A4A9A5805
:1068800082600A4A9A58C260094A9A580261094AC3
:106890009A584261084A9A588261084A9B58C361D3
:1068A0007047C046F80A0208047800000878000023
:1068B0000C780000107800001478000018780000B0
:1068C0001A4B1B681A008832196812688A18016A04
:1068D00011601A008C32196812688A18416A1160B6
:1068E0001A0046321278002A1ED09A68E0321268E6
:1068F000D20619D5F0224168DB68D201995081682F
:106900000B4A9950C1680B4A995001690A4A99503B
:1069100041690A4A99508169094A9950C169094AED
:1069200099500168E83299507047C046F80A020849
:1069300004780000087800000C780000107800004F
:106940001478000018780000F7B50700FFF73AFD4B
:10695000664D06006B68002B00D07DE0F9F7BDFDA9
:106960006B680090002B00D089E0614C2268130016
:10697000BA33198807234B43126A9B181A68002AF6
:10698000FCDADB68DA0021D51B0F1B07594801939D
:10699000FFF752FF5849212E00D075E02268902061
:1069A000130088331C68136800011C1923680B400E
:1069B0000343236013008C3312681B68D3181A68D2
:1069C0001140084318604B4B019A13438022484EF4
:1069D0009205316813430A00BA3210880722002456
:1069E0004243096A5218D36054605368FFF7F3FCBE
:1069F00080235B0098425DD1380002F0ADF8326828
:106A00001300BA33198807234B43126A9B181A687C
:106A1000002AFCDADF68FB0003D538010009FFF724
:106A20004FFF364B32681F401300BA3319880723D3
:106A30004B43126A00989B180022DF605A60F9F7F6
:106A400050FD002C0FD16B68002B03D008210120D2
:106A5000FFF7FAFD2000FEBD01210800FFF7F4FD5D
:106A6000041E00D17AE76B68002B03D002210120BD
:106A7000FFF7EAFD224B9C42ECD0224CEAE70421CE
:106A80000120FFF7E1FD70E72068802203008833D2
:106A90001C68036852001C1923680B4013432360D1
:106AA00003008C3300681B68C318186801400A4350
:106AB0001A6088E733681A00BC32196A12685218E3
:106AC0001168002910DBBA331B889A181368002B51
:106AD0000ADB04230C4A11690B431361012F01D017
:106AE00030BF8CE720BF8AE7054C88E7980702088B
:106AF000F80A020858070208FF00FFFFFFFFFFDF48
:106B000005004200FF00420000ED00E010B5002843
:106B100010D107292BD8174B89001C682300B433E8
:106B20001B8824681B19591803231340124A1A435F
:106B30000A6010BD01280DD10E4B19680B00B63349
:106B400009681B885B18032111400B4A0A431A602D
:106B50000020EEE702280AD1064B19680B00B83373
:106B600009681B885B1803210A400349EEE70348C4
:106B7000DFE7C046F80A02080000FA0501004200FB
:106B800010B5002811D1184B1A681300B4331C88B3
:106B900003230B40154919431368E3181B180430ED
:106BA00019602028F8D1002010BD01280CD10E4B0F
:106BB0001A681300B63312681B889B1803220A4018
:106BC0000A4911431960EEE702280AD1064B1A68F8
:106BD0001300B83312681B889B1803221140034A24
:106BE000EFE70348E0E7C046F80A02080000FA05AC
:106BF00001004200024B58694000C00F7047C04678
:106C00000000264010B50D4B1B6847331B78002B46
:106C100012D0FFF7EFFF0A4B002804D180225969F8
:106C2000D2050A435A6180229620996912060A43C6
:106C30009A618000FFF714FB10BDC046F80A0208F5
:106C4000000026400020064B1B6847331B78834218
:106C500003D0044B986907231840C0B27047C04660
:106C6000F80A02080000264070B50D4B04001B68AE
:106C70000D0047331B78002B11D0FFF7E3FFA04234
:106C80000DD0072207498B699343224013438B6140
:106C9000002D04D0A04202D2C820FFF7E1FA70BD57
:106CA000F80A020800002640054B1B6847331B7892
:106CB000002B04D0034A93695B005B089361704723
:106CC000F80A02080000264010B50400FFF792FF02
:106CD0000A4B1B6847331B78002B09D0002807D0CC
:106CE000074B002C05D080229969D2050A439A618E
:106CF00010BD9A6903490A40F9E7C046F80A02083C
:106D000000002640FFFFFFBF074A084BD058B022C3
:106D1000E8235205DB00D35C1F221040C01A431E3B
:106D20009841C0B27047C046000026401CFF0000DA
:106D30000120024B1B68DB0D984370470000264082
:106D400010B5114C23689B061CD5FFF7F1FF226894
:106D5000002813D00D4B13432360FFF7D5FF012804
:106D600002D150220A4BE2500120FFF779FA80232A
:106D700000202268DB051343236010BD054B13433D
:106D80002360F1E70448F8E70000264000000417FC
:106D9000307F0000000004160400420010B5FFF729
:106DA000C7FF184C236800280DD0174A13402360F2
:106DB0000820FFF755FA64232268002A07DB002B1E
:106DC00003D1124811E0124AF0E7013BF4E7002B2F
:106DD000F7D023680F4A012013402360FFF740FAE1
:106DE000FFF7A6FF002801D1002010BDFFF78CFFA0
:106DF0000128F9D1B022084B5205D258074BE25076
:106E0000F2E7C04600002640FFFFFBAC0200420054
:106E1000FFFFFBADFFFFFFFB10180000307F0000FD
:106E200010B5FFF785FF431E9841802340425B0465
:106E30001840054BC018054B1B680340181A434205
:106E40005841C0B210BDC0460000045200002640A8
:106E5000F7B50700FFF7B6FB002848D0F9F73DFB70
:106E6000B0240190234D244E6405002F1CD1E8234B
:106E7000AF51DB000120E45CFFF73EFCE4B2061EEC
:106E80000DD1FFF7B3FA1F211C4A0C40AB588B43BE
:106E90001C43AC50002F20D1FFF722FB3E0001988D
:106EA000F9F71FFB3000FEBDFFF7BAFF50230028A3
:106EB00001D1134BE3581F22AB511049114B032052
:106EC000E45C6B58E4B293431A000B2313436B50FA
:106ED000FFF7C6F9FFF7CAFAD5E70720FFF7C0F9B1
:106EE000FFF730FB0020FFF707FC0600D7E7064E50
:106EF000D8E7C04600002640307F00001CFF00009D
:106F0000101800004107000003004200F8B505001A
:106F1000FFF70EFF002857D0F9F7DFFA0600022D21
:106F20003CD1FFF7F1FE00282ED11F222C482D491D
:106F3000435893431A000B23134343500920FFF790
:106F40008FF9E023264FDB033A68E1201343072241
:106F50003B607B69154093431D4380237D617A69C3
:106F6000DB0513437B6180237A691B0613437B6136
:106F70008000FFF775F9802300243A681B0413434F
:106F80003B60194BFC5004E00020FFF761FF041E3A
:106F9000CBD03000F9F7A5FA2000F8BD052D11D1AE
:106FA000FFF7B2FE012807D11F220D480D494358B3
:106FB00093431A001B23BFE70120FFF749FF041E7C
:106FC000F2D0E6E7094CE4E70722054B04005B69D1
:106FD00013409D42E0D02800FFF7ECFB0400DBE704
:106FE000000026401CFF0000307F0000030042002C
:106FF000054A536C1B0ADBB23A2B03D1516C034B8D
:107000000B4353647047C04600002740003A0020FD
:10701000064A536C1B0ADBB23A2B06D1536C044967
:107020001940E8239B010B4353647047000027403D
:10703000FFC5FFDF0449054A4B6C1A40E8239B015A
:1070400013434B647047C04600002740FF00FFFF1A
:10705000C022C0230349520088581B0603438B50AB
:107060007047C04600002640C023044A5B00D05849
:10707000800F431E9841C0B27047C04600002640B2
:10708000C0228020064952008B58C0059B009B08F7
:1070900003438B50802388581B0603438B50704753
:1070A0000000264010B50400FFF7DEFF002808D1DD
:1070B000C423044A5B00D058A4B2000C000420434F
:1070C000D05010BD0000264010B50400FFF7CCFFE3
:1070D00000280BD1C422F0200549520000032404EB
:1070E0008B580440034803401C438C5010BDC046DD
:1070F00000002640FFFFF0FFE0230121024ADB00F1
:10710000D150D3587047C0460000264010B51148F2
:10711000FAF700FFFFF7B4FFC02201200E4952002A
:107120008B5883438B5000F07DF80C4A802103205C
:10713000FBF74CF90A48FBF71FF80A4B1B68513361
:107140001B78002B02D00848FBF752F8FCF722FD11
:1071500010BDC046708F0010000026400C000008D3
:107160006C090208F80A020830900010F0B50025FA
:1071700085B00395FFF7CAFF62B6FAF7B1FE80202B
:1071800002AA03A94000FAF747FD1E4C1E4B1F4EF2
:107190000093019533001E4A21000398F9F7F8FD8A
:1071A000230048331B78AB4228D08022E36CD20006
:1071B0009D18184B676B1E60FCF786FD637E012BE4
:1071C00006D1637C002B03D0216AE069F9F762FDE8
:1071D000230038331E78002E04D0E06BFAF71CFE33
:1071E000FAF78EFE06210E20FDF7D0FF28003200B0
:1071F0003900FAF7B3FD002005B0F0BD8022E36945
:107200005202D5E7AC070208940F02082C090208C5
:10721000181002083C07020810B50020FBF78EF892
:1072200010BD000010B50020FEF744FF041E25D05D
:10723000134B1860FEF7B8F8411C200000F08CF8E2
:10724000104B04001860FDF7DDFF411C200000F02A
:1072500083F80D4B441E18600C49200000F07CF8A8
:10726000FA210B4B013018708900200000F074F8EF
:10727000084B01301860084BC003186010BDC046B1
:10728000F8000208FC000208F400020840420F0067
:107290000801020804010208000102089023034AC1
:1072A0005B01D058032318407047C04600002040BF
:1072B00010B59024F9F711F9074B64011A590749E1
:1072C0001140074A0A431A51102259681142FCD052
:1072D000F9F707F910BDC04600002040FCFF000090
:1072E0000100FA05F8B590250E4C6D010700F9F77D
:1072F000F4F863590600DB439B0701D1FFF7D8FF81
:1073000080239B00E7506359074A1A40074B1343F9
:107310006351102362681A42FCD03000F9F7E1F89B
:10732000F8BDC04600002040FCFF00000300FA0545
:1073300002B4714649084900095C49008E4402BC08
:107340007047C04603B47146490840004900095AD5
:1073500049008E4403BC7047002243088B4274D31B
:1073600003098B425FD3030A8B4244D3030B8B4246
:1073700028D3030C8B420DD3FF22090212BA030C4F
:107380008B4202D31212090265D0030B8B4219D330
:1073900000E0090AC30B8B4201D3CB03C01A524150
:1073A000830B8B4201D38B03C01A5241430B8B4298
:1073B00001D34B03C01A5241030B8B4201D30B0381
:1073C000C01A5241C30A8B4201D3CB02C01A5241A8
:1073D000830A8B4201D38B02C01A5241430A8B426B
:1073E00001D34B02C01A5241030A8B4201D30B0254
:1073F000C01A5241CDD2C3098B4201D3CB01C01A6E
:10740000524183098B4201D38B01C01A5241430977
:107410008B4201D34B01C01A524103098B4201D365
:107420000B01C01A5241C3088B4201D3CB00C01AD2
:10743000524183088B4201D38B00C01A524143084A
:107440008B4201D34B00C01A5241411A00D201466F
:10745000524110467047FFE701B5002000F006F8E2
:1074600002BDC0460029F7D076E770477047C04696
:10747000002B11D1002A0FD1002900D1002802D001
:107480000021C943081C07B4024802A14018029019
:1074900003BDC046D9FFFFFF03B4684601B502989B
:1074A00000F04EF8019B9E4602B00CBC7047C046EF
:1074B000F0B5CE46474615042D0C2E0080B50704C6
:1074C000140C3F0C9946030C7E435D4367436343B2
:1074D0007F19340CE4199C46A54203D980235B0232
:1074E0009846C4444B4643435143250C36046544F7
:1074F000360C2404A4195B19591820000CBC9046C2
:107500009946F0BD70B500220C4B04000D0000F050
:10751000C7FF002804D12000290000F01DFF70BD26
:10752000064B00222000290000F0CEFB00F014FFE3
:1075300080231B069C466044F1E7C0460000E04102
:10754000F0B54F464646D646C0B5040082B00D00A1
:10755000914698468B422FD82CD04146484600F0A1
:10756000C7FF29000600200000F0C2FF331A9C4626
:10757000203B9A4600D576E04B46524693401F008A
:107580004B46624693401E00AF4228D825D0534652
:10759000A41BBD41002B00DA7BE0002200230092F7
:1075A0000193012352469340019301236246934085
:1075B000009318E08242D0D9002200230092019368
:1075C0000A9B002B01D01C605D600098019902B0FD
:1075D0001CBC90469946A246F0BDA342D7D90022D2
:1075E0000023009201936346002BE9D0FB079846E5
:1075F000414672080A437B0866460EE0AB4201D161
:10760000A2420CD8A41A9D41012024196D410021E9
:10761000013E24184D41002E06D0AB42EED9013E6A
:1076200024196D41002EF8D1009801995346001994
:107630006941002B23DB2B005246D3402A006446CD
:10764000E2401C0053461500002B2DDB2600574658
:10765000BE40330026006746BE403200801A994182
:1076600000900191ACE7624620239B1A4A46DA401B
:107670006146130042468A4017001F4380E7624676
:1076800020239B1A2A0066469A402300F3401343A6
:10769000D4E76246202300219B1A00220091019228
:1076A0000122DA40019280E72023624626009B1ADD
:1076B000DE402F00B0466646B74046463B003343A7
:1076C000C8E7C046F0B55746DE464E464546E0B5EB
:1076D000834607000E03480085B092461C00360B17
:1076E000400DCD0F002800D19DE0954B984239D038
:1076F0008023F6001B041E43924A7B0F33439946B6
:10770000944603006344009300230026FF00029385
:1077100023031B0B98466300E40F52465B0D019454
:1077200000D1B3E086498B4200D19EE04246D100B1
:10773000802212040A435146490F11438B46814966
:1077400052468C4600996344CB1A0021D200009324
:107750002B0063409A460F2E00D905E17A4BB60004
:107760009B599F465B463343994600D0B8E00223BD
:107770000826002700900293CAE7CB463A000299F8
:107780000195019B9A46022927D0032900D180E266
:10779000012944D06D49009B8C4663441C00002C99
:1077A00038DD530700D013E2D2085B46DB0109D570
:1077B0005946674B19408B468021C9008C46009B77
:1077C00063441C00634B9C4207DC5B4664055F0717
:1077D0005B0217431B0B620D02E000230027584A8F
:1077E00000211B031C0B0B0D1B05234314055A4AD8
:1077F000380013401C4353466400DB0764081C43F5
:10780000210005B03CBC90469946A246AB46F0BD6F
:107810000122524201231B1B382B00DCADE1002268
:1078200000230027DCE75B46334399465ED0002EF9
:1078300000D18AE1300000F03DFE03000B3B1C2B21
:1078400000DD7BE11D22D31A5A460100DA400839D7
:107850008E4013005F46334399468F403F4B0026CE
:107860001B1A00930023029352E7414653460B43F1
:107870003B499B468C46009B634400935B46002B30
:107880003BD1022300221E43022161E743461343FA
:107890009B4637D04346002B00D162E1404600F0C2
:1078A00009FE03000B3B1C2B00DD53E102004146A7
:1078B000083A914088461D21CB1A5146D9400B0009
:1078C00041460B439B46534693401A00009B254973
:1078D0009C46604403008C4663440093002137E7D4
:1078E0000323B14600900C26029311E70023009376
:1078F00001330426002702930AE70323C3461E43ED
:10790000032125E701331E430022012120E7002344
:107910009A46802300271B03094A61E780234946D2
:107920001B03194200D1E2E05946194200D0DEE0C3
:107930000B431B0317001B0BA246014A50E7C0462E
:10794000FF07000001FCFFFF64900010FF03000030
:10795000FFFFFFFEFE070000FFFF0F800DFCFFFF93
:1079600001F8FFFFF3030000D94500D9CBE000D1B7
:10797000C6E03C0048460027009B013B00935B4665
:10798000160E1B021E431302984633041B0C994625
:10799000310C0191FFF766FD4A4642430B04210C6E
:1079A000050019438A4207D98919013D8E4203D83F
:1079B0008A4201D9851E8919881A0199FFF752FD5B
:1079C00009048C464A46210464464243090C0300DC
:1079D00021438A4204D98919013B8E4200D8F1E043
:1079E0002D041D43AB464346891A4246280C120417
:1079F0001D0C5B46140C22001B041B0C5A43039401
:107A00006B434443029568431B19150CEB189C42C9
:107A100003D980246402A44660441C0C15041B0492
:107A20002D0C20185D19814277D373D00C1AA24A0D
:107A30007D1BAF42BF419446009B7F426344E01BE5
:107A40001C00864200D1DBE00199FFF70BFD4A469E
:107A500042430B04290C070019438A4207D98919AC
:107A6000013F8E4203D88A4201D9871E8919881A9C
:107A70000199FFF7F7FC09044A46894629044D4657
:107A80004243090C030029438A4207D98919013B63
:107A90008E4203D88A4201D9831E89193F04891A6C
:107AA0003A00039F1A43380013041B0C58438146C5
:107AB0000298150C6F43434345434846000C8446E7
:107AC000DB1963449F4203D9802040028446654409
:107AD00048461F0C00041B04000C7D191818A9420D
:107AE00000D284E000D17FE001231A4357E68023CF
:107AF0004A461B0313431B031B0BAA466F4A6FE640
:107B0000BA4200D935E74B46DC0758087B081C43CE
:107B1000FF0734E70024AF4289D247444745A441D8
:107B20005B466442A4196418013BA6421ED2A042DF
:107B30006DD800D1B6E0241A9B4678E703005A4678
:107B4000283B9A400027914688E6584600F0B2FC50
:107B5000203072E603005246283B9A4093460022AA
:107B6000B4E6504600F0A6FC20309AE6A642E2D1E8
:107B7000B845DCD9341A9B4659E71F2B65DC504CBD
:107B80000099A4465C46614408008C401100824084
:107B9000D940501E82410C4314435A46DA40130028
:107BA000620709D00F222240042A05D02200141DAA
:107BB0009442894149425B181A0262D5012200238E
:107BC00000270DE68A4200D80AE7831E891907E7D5
:107BD0000F231340042B00D1E6E5171D9742924175
:107BE00053429B44FA08E0E5002800D1D7E571181C
:107BF000531EB14227D3A94215D358D01A0073E7B8
:107C0000002B00DC04E6012300229B44CDE5022387
:107C10004744474589415B429C46494289190C19B2
:107C2000E344241A03E743465F0047459B41B846B7
:107C30005B429E19023A8919A94200D054E7404597
:107C400000D051E7ABE51A00F6E71F215F46494235
:107C50000C1BE740202B07D01A49009B8C4663443D
:107C600018005B4683401A43501E82413A4307275F
:107C70000023174009D00F210023114014000429CC
:107C800095D122005F075B021B0BD208174300222D
:107C9000A6E5802359461B030B431B0317001B0B50
:107CA000064A9DE5BD42B2D89B460024BFE680450A
:107CB000B9D31A00C3E7C046FF030000FF07000066
:107CC0001E0400003E040000F8B557464E464546E7
:107CD000DE460C000903E0B5490A460F5F00314358
:107CE0001E03DB0F760A9B46530F3343C84E6500D5
:107CF000C000E40FD2006D0DA24681467F0D9C4668
:107D00009046B74200D1B9E05B46012673409B46DE
:107D1000EE1BA34500D183E0002E63DD002F00D0D1
:107D2000B1E06346134300D123E1731E002B00D062
:107D3000BAE1861A6346B04280410125C91A404221
:107D4000091A0B0200D447E149024B0A9846434600
:107D5000002B00D189E1404600F0ACFB0300083B5A
:107D60001F2B00DD7CE120223000D21A4146D0409A
:107D7000994002009E400A439D4200DD6AE15D1B7E
:107D80006B1C1F2B00DD94E1202110003500C91A67
:107D90008E40DA408840DD40711E8E41110007227E
:107DA0002843002506433240002A09D00F233340E0
:107DB000042B05D0331DB342B641764289191E000B
:107DC0000B0200D43DE26A1C914B55056D0D9A42A1
:107DD00000D119E18F4AF6080A405707520237438B
:107DE000120B9BE0002E00D0C5E06E1C7605760DD0
:107DF000012E00DC48E16746861ACB1BB042BF412A
:107E00007F42B8461F004346FF1A3B00B8461B029C
:107E100000D55FE137439AD100220024002579E0A4
:107E2000002E00DCFAE0002F00D18DE0784B9D425F
:107E300067D0802367461B041F43BC46382E00DCF6
:107E400052E1634613435A1E93411E1886428041F5
:107E5000404209180B0200D4BEE06D4B01359D4233
:107E600000D1D2E06B4A73080A4001210E401E4344
:107E70005108D30707221E43324095E71E001643E0
:107E800000D045E740E7624B9D423AD080236746E9
:107E90001B041F43BC46382E00DDEBE01F2E00DC28
:107EA0003AE133006746203BDF403B00202E05D0FF
:107EB0004027BF1B6646BE40324390464646721E70
:107EC00096413343DAE0002B00D114E263461343BA
:107ED00000D168E180234E07C008C9081B03064390
:107EE000194208D06046C008184204D16346010018
:107EF000D2085E071643F3009946C900720F444D3D
:107F000011434B46DE08424B4F073743CA089D4298
:107F100000D16EE012036D05120B6D0D00211203EE
:107F2000130B0A0D12051A433B4B2D0513402B432F
:107F30005B00E4075B082343380019003CBC904613
:107F40009946A246AB46F8BD6346134311D0731E53
:107F5000002B00D007E186188642804161444042F0
:107F6000091801250B0237D502257BE73E00614643
:107F700091463500C5E75C46002D00D0E1E00B00DE
:107F80000343F3D0731C00D1ACE1214B9F4200D1DD
:107F90003AE1F343382B00DD6FE11F2B00DD8CE16C
:107FA00020250E00ED1AAE40B0460600AA46DE407F
:107FB000454635432E005546D940A8406346451EE8
:107FC000A8415B1A9C463043161AB242924163465E
:107FD0005242991A3D00B4E607223240002A00D0EE
:107FE000E4E60B4BF6084F073743CA089D4200D022
:107FF00090E73B00134300D1A6E180231B031A4303
:108000001203120B024D89E715000022002785E7B5
:10801000FF070000FFFF7FFFFFFF0F80002E00D053
:10802000C7E06B1C5E05760D012E00DCF0E0C84D4C
:10803000AB4200D1B9E085180A008542894162440B
:10804000494251180722CE076D082E434908324095
:108050001D00A9E6BF49ED1A114007223240A3E6F0
:10806000320028388240002686E6300000F022FAEE
:10807000203073E6634613435A1E9341C61AB0423A
:1080800080414042091A5CE60E00674606431743EA
:10809000002D5ED1002E00D0F3E0002F00D11EE1B4
:1080A0005C46614691462CE7A94FBE427BD01E003C
:1080B000F1E610001F3DE840202B03D04021CB1AF1
:1080C0009A401643731E9E41072206433240002108
:1080D000002583E7161A6346B2428041591A40428E
:1080E0000B1A98465C4632E61F2E00DDABE02027D7
:1080F000BB1B9A4663465746BB40994613004F4602
:10810000F3401F433B005746BA40571EBA41134342
:108110006246F240891898E62027BB1B9A466346C0
:108120005746BB40994613004F46F3401F433B0060
:108130005746BA40571EBA4113436246F240891A65
:108140009CE7834B9F425FD080252D0473422943D7
:1081500020E7002E0CD1002F00D1D0E05C46614614
:1081600091467B4DCDE67A4FBE421CD01E0065E69F
:10817000002F18D0C0084E0706438020C90800030E
:10818000014208D06346DC08044204D12100DA46EB
:10819000D2085E071643F300994601245346C900EE
:1081A000720F11431C406A4DABE61D0000220027F0
:1081B000B4E6002D59D10B00034300D1D6E6731C61
:1081C00000D1B2E0624B9F421ED0F343382B6FDCEC
:1081D0001F2B00DD97E020250E00ED1AAE40B046C3
:1081E0000600AA46DE40454635432E005546A840C7
:1081F000D940451EA8418C440643B6189642924188
:10820000514261443D0025E63D006146914678E6D5
:108210000B000343002D00D055E6002BF5D063463C
:10822000134300D16DE68618864280416144404286
:10823000091800220B0200D4D0E6464B0135194044
:10824000B2E5B1465DE633006746203BDF403B00C8
:10825000202E05D04027BF1B6646BE4032439046C5
:108260004646721E96413343EFE5394B9F42CBD0D1
:1082700080252D0473422943A8E70843411E884105
:10828000A2E6002F00D13CE66346861ACF1AB04220
:108290009B415B42FB1A98461B024ED5161A634659
:1082A000B2429241591A5242891A5C4600227BE539
:1082B00001430E00711E8E419FE71D000E00203D00
:1082C000EE40B046202B04D04025EB1A99400843DD
:1082D000814648464346411E8841184374E60022C1
:1082E000002417E6161A6346B2429241591A5242C6
:1082F000891A3D0025E561469146154D01E680222B
:108300000024120379E61D000E00203DEE40B04629
:10831000202B04D04025EB1A9940084381464E4655
:108320004346711E8E411E4367E7861896429B4165
:1083300061445B42C9183D008CE547463743CED0C7
:1083400007224146324049E600273A00E6E5C046AA
:10835000FF070000FFFF7FFF30B5144D0A034B00FD
:10836000120B5B0DC90F0024AB4211DD104CA34270
:1083700010DC8024640322430E4CE41A1F2C0CDD15
:108380000D48C31ADA4013005C42002900D11C00DA
:10839000200030BD094BCC18FAE7094DE040AC464F
:1083A00063449A4013000343EEE7C046FE03000017
:1083B0001D0400003304000013040000FFFFFF7FD2
:1083C000EDFBFFFF70B500282DD0C317C5185D4029
:1083D000C40F280000F06EF8154B1B1A5B055B0DEF
:1083E0000A2815DD0B38854000222D032D0B0021B6
:1083F00010002D030A0D2D0B12052A430D4D1B05F0
:108400002A4013435B00E4075B082343190070BD57
:1084100002002900153291400A000B21081AC540BC
:108420002D032D0BE3E70024002300250022DEE7C7
:108430001E040000FFFF0F808446101C62468C461D
:10844000191C634600E0C0461FB500F0FDF8002887
:1084500001D40021C8421FBD10B500F055F84042BC
:10846000013010BD10B500F0EFF8002801DB00204E
:1084700010BD012010BDC04610B500F0E5F8002881
:1084800001DD002010BD012010BDC04610B500F078
:1084900077F8002801DC002010BD012010BDC04687
:1084A00010B500F06DF8002801DA002010BD0120A1
:1084B00010BDC0461C2101231B04984201D3000CAF
:1084C00010391B0A984201D3000A08391B09984247
:1084D00001D30009043902A2105C40187047C0465D
:1084E000040302020101010100000000000000007D
:1084F00010B5002903D1FFF7DDFF203002E0081C92
:10850000FFF7D8FF10BDC046F0B54F464646D646E9
:108510008446C0B58046194E18030F034D00000B6A
:108520005C0082463F0B6D0DC90F9146640DDB0F59
:108530000120B5420AD0B44203D0A54201D157452B
:108540000CD01CBC90469946A246F0BD66463E4300
:10855000F7D1AC42F5D154461443F2D10120C845BD
:10856000EFD1994207D0002DEBD163461F4338006D
:10857000471EB841E5E70020E3E7C046FF070000DB
:10858000F0B54F464646D6464D00C0B50E03C90F5E
:108590008A462C491F035C008046360B6D0D9146C0
:1085A0003F0B640DDB0F8D421ED08C4216D0002D88
:1085B0001ED130438446002C01D13A4323D0624679
:1085C000002A1AD09A4529D0514602200139084084
:1085D00001381CBC90469946A246F0BD39001143B3
:1085E000E5D002204042F4E73043FAD1AC420FD04C
:1085F000002C0FD13A43E7D00CE00122013B93431A
:1086000018000130E5E763460020002BE1D0DBE7EE
:108610003A43E6D19A45D7D1A542D5DCA54205DB40
:10862000BE42D1D808D00020BE42D2D2504601234B
:10863000013898430130CCE7C845C5D80020C8456B
:10864000F4D3C6E7FF070000F0B54F464646D646CE
:108650004D00C0B50E03C90F8A462E491F035C00AA
:108660008046360B6D0D91463F0B640DDB0F8D423E
:1086700018D08C4211D0002D18D130438446002CE4
:108680001ED13A431CD163460020002B30D0514606
:1086900002200139084001382AE039001143EAD0AC
:1086A000022025E03043FBD1AC4226D0002C26D15D
:1086B0003A4324D15146022001390840013817E0DD
:1086C0006246002A0FD09A45E1D1A54205DBBE42A1
:1086D000DDD819D00020BE420AD25046012301380D
:1086E0009843013004E00122013B9343180001301C
:1086F0001CBC90469946A246F0BD3A43D0D19A455B
:10870000C5D1A542C3DCE0E7C845C0D80020C845B4
:10871000E3D3EDE7FF070000EC300068704700008E
:1087200010B5034B0100186800F07CF810BDC0467E
:108730000C01020810B5034B0100186800F028F87E
:1087400010BDC0460C01020882B0002900D101A969
:10875000101E06D0002B06D013780B601078431E35
:10876000984102B0704702204042FAE7002310B55A
:108770009A4200D110BDCC5CC4540133F8E7030029
:108780001218934200D1704719700133F9E70000C5
:1087900070B50500002910D00C1F2368002B00DAEB
:1087A000E418280000F0ACF91D4A1368002B05D12D
:1087B00063601460280000F0A4F970BDA34209D9D9
:1087C000216860188342F3D118685B684118216002
:1087D000EEE713005A68002A01D0A242F9D91968BD
:1087E0005818A0420BD12068091858181960824205
:1087F000E0D110685268411819605A60DAE7A04267
:1088000002D90C232B60D5E721686018824203D17E
:10881000106852684118216062605C60CAE7C04617
:10882000EC0A0208032370B5CD1C9D4308350600F1
:108830000C2D1ED20C25A9421DD8300000F060F985
:10884000254A14682100002919D1244C2368002BE3
:1088500003D1300000F044F820602900300000F01F
:108860003FF8431C2BD10C233000336000F049F952
:1088700003E0002DDFDA0C233360002070BD0B68AD
:108880005B1B19D40B2B03D90B60CC18256003E0BC
:108890004B688C420DD11360300000F032F920009B
:1088A00007220B30231D9043C31AE7D05A42E250EF
:1088B000E4E763600C00EFE70C004968C3E70323BB
:1088C000C41C9C43A042E1D0211A300000F008F8FB
:1088D000431CDBD1C7E7C046EC0A0208F00A0208D5
:1088E000002370B5064C05000800236000F00AF96B
:1088F000431C03D12368002B00D02B6070BDC04601
:1089000020100208C9B20378002B04D08B4200D19A
:1089100070470130F7E74B42594149420840F7E7B9
:1089200002780B78002A03D0013001319A42F7D047
:10893000D01A704703000A7801311A700133002AF7
:10894000F9D17047002330B59A420AD0013AC45C8D
:10895000CD5CAC4204D1934202D00133002CF6D15D
:10896000631B180030BD0000F0B51F000E008DB075
:108970000B900291039212983478FFF7CDFE0822F3
:1089800000194378751C134053D12D2C53D17478A2
:10899000B51C01330193002F00D18AE0102F0AD1BA
:1089A000302C08D120222B789343582B00D07AE02A
:1089B00010276C780235019B002B41D1013B0493B9
:1089C0003E4B05933A00FB17049805990893FEF770
:1089D0004FFD002309900E00002000210A92220082
:1089E000303A092A31D81400A7423DDD5A1C1DD067
:1089F000B14236D802D1099B984232D8099B8342B2
:108A000006D18E4204D101230A9A5B42A2420DDBB9
:108A10000B00020008993800FEF74AFDE3170694A0
:108A20000793069B079CC018614101232C780135F0
:108A3000D5E72E009FE72B2CACD1B51C7478A9E7A5
:108A40000023049380231B06BBE72200413A192A26
:108A500001D8373CC8E72200613A192A04D8573CAC
:108A6000C2E701235B42E1E75A1C09D10B9A233389
:108A70001360039B04980599002B0ED10DB0F0BD37
:108A8000019A002A04D006000F0000217042B9416B
:108A9000039A002AF2D0002B01D06B1E0293039B95
:108AA000029A1A60EAE73024002F00D083E70827F3
:108AB00081E7302C00D175E70A277CE7FFFFFF7FB5
:108AC00037B51300064A05001068046A002C00D16F
:108AD000044C0A0000942900FFF746FF03B030BDA4
:108AE0000C010208700102080B1E04D0FF2A04D9F1
:108AF0008A2303608B3B180070470A700123FAE752
:108B000070477047044A1368002B00D1034B1818B4
:108B1000106018007047C046F40A020828100208C6
:108B2000F8B5C046F8BC08BC9E467047F8B5C046CC
:108B3000F8BC08BC9E46704701B40248844601BC9C
:108B4000604700BF7D03020801B40248844601BCAF
:108B5000604700BFE502020801B40248844601BC38
:108B6000604700BFA90402084142434445464748C4
:108B7000494A4B4C4D4E4F505152535455565758ED
:108B8000595A6162636465666768696A6B6C6D6E89
:108B90006F707172737475767778797A3031323399
:108BA000343536373839006E756C6C0066616C731D
:108BB000650074727565007265736F7572636573B5
:108BC00000616464726573730073697A650053436E
:108BD0005241544348006C61756E63680061637173
:108BE0005F77696E007764745F656E61626C6500C3
:108BF0007764745F74696D656F7574007570677202
:108C00006164655F6D6F64650073776170006D7599
:108C10006C74695F696D616765006D6F6E6F746F0D
:108C20006E696300424F4F540055504752414445CE
:108C300000656E637279707400656E63727970742A
:108C40005F6B65795F696400626F6F745F617574F3
:108C50006800736D69665F6964007365745F696D50
:108C6000675F6F6B005354415455535F50415254EA
:108C70004954494F4E006D34007065726D697373CD
:108C8000696F6E00636F6E74726F6C006B65790054
:108C9000657874436C6B456E61626C6500657874D1
:108CA000436C6B46726571487A00657874436C6BEF
:108CB000506F727400657874436C6B50696E4E75BA
:108CC0006D0065636F456E61626C650065636F463C
:108CD000726571487A0065636F4C6F61640065630B
:108CE0006F4573720065636F44726976654C657693
:108CF000656C0065636F496E506F72740065636FD9
:108D00004F7574506F72740065636F496E50696E71
:108D10004E756D0065636F4F757450696E4E756D5D
:108D20000077636F456E61626C6500627970617394
:108D300073456E61626C650077636F496E506F7248
:108D4000740077636F4F7574506F72740077636F40
:108D5000496E50696E4E756D0077636F4F75745034
:108D6000696E4E756D00657874636C6B007072652A
:108D700073656E74006669726D7761726500636514
:108D8000727469666963617465006F70656E006412
:108D9000697361626C656400656E61626C65640034
:108DA000616C6C6F77656400646562756700626F03
:108DB0006F745F75706772616465007372616D7066
:108DC00077726D6F6465006D6163726F4E756D00D3
:108DD00074797065006172726179006974656D7390
:108DE000006E756D62657200696E7465676572000C
:108DF000626F6F6C65616E00737472696E67006D8F
:108E00006178696D756D006D696E696D756D007362
:108E100072616D3000464C4153485F5043315F539F
:108E2000504D00464C4153485F50433200464C4140
:108E300053485F50433300464C4153485F504334DE
:108E400000464C4153485F4D41494E5F434F4445B6
:108E500000464C4153485F4D41494E5F584F0046D4
:108E60004C4153485F4D41494E5F44415441004697
:108E70004C4153485F53555045525649534F5259F0
:108E800000464C4153485F574F524B5F5345435543
:108E9000524500464C4153485F574F524B00535286
:108EA000414D5F5043305F50524956005352414D3F
:108EB0005F5043305F505542005352414D5F535015
:108EC0004D5F50524956005352414D5F53504D5FD4
:108ED000505542005352414D5F5043315F5052490B
:108EE00056005352414D5F5043325F505249560035
:108EF0005352414D5F5043335F50524956005352D5
:108F0000414D5F5043345F50524956005352414DDA
:108F10005F4D41494E005352414D5F444150005313
:108F20004D49465F434F444500534D49465F584FB6
:108F300000534D49465F444154410000A10FB90B15
:108F4000D107DC05E903EE02F5017701FB00BC0067
:108F50007E005E003F002F002000180010000C0073
:108F600008000600040003000200020001000100E6
:108F700000002040000024400000004000000000ED
:108F800000002340000030400000314000009F40BE
:108F9000000022400000104000009D4020202020C2
:108FA00020131010101D208017007500FF0305010D
:108FB00005001C03100000003FC00000000400007A
:108FC000000000000019324B647D000000000080AA
:108FD0004000080B100000000000FF012002001FED
:108FE00000800004FF081018001000140018001C76
:108FF0004044484C500000000810000008000000E9
:109000000400000004100000001200000421000011
:10901000002100000016000040114002C41300139C
:109020008013A01340138813A81320001C00000015
:10903000030000000100000001000000000000002B
:1090400005036000040000000100000000000000B3
:10905000010000000604600008000000CC0A0208BD
:109060001972001068790010DA7700101E7800106D
:10907000827700101E7800100E7900101E78001004
:1090800082770010DA770010DA7700100E7900107E
:10909000827700107A7700107A7700107A770010C4
:1090A0001C7900104300504F534958002E000020F7
:1090B0002020202020202020282828282820202088
:1090C0002020202020202020202020202020208838
:1090D000101010101010101010101010101010049C
:1090E00004040404040404040410101010101010EC
:1090F00041414141414101010101010101010101E0
:1091000001010101010101010101101010101010F5
:1091100042424242424202020202020202020202AF
:1091200002020202020202020202101010102000CB
:10913000000000000000000000000000000000002F
:10914000000000000000000000000000000000001F
:10915000000000000000000000000000000000000F
:1091600000000000000000000000000000000000FF
:1091700000000000000000000000000000000000EF
:1091800000000000000000000000000000000000DF
:1091900000000000000000000000000000000000CF
:1091A00000000000000000000000000000000000BF
:0491B00000000000BB
:0891B4008CE3FF7F01000000C5
:1091BC00000400100000020880000000DC91001088
:0891CC008000020860050000AC
:0891D40000060208240A000055
:1091DC003587001021870010158E0010238E00108B
:1091EC002D8E0010378E0010418E0010518E001005
:1091FC005F8E00106F8E0010818E0010938E001009
:10920C009E8E0010AC8E0010B98E0010C78E001010
:10921C00D48E0010E28E0010F08E0010FE8E001026
:10922C000C8F0010168F00101F8F0010298F00104C
:10923C00318F0010248C0010298C0010658C0010CC
:10924C00CE8B001000093D0000127A0000093D0091
:10925C000000D007A00F000004000000100102085D
:10926C0000000000000000000000000000000000F2
:10927C0000000000000000000000000000000000E2
:10928C0000000000000000000000000000000000D2
:10929C0000000000000000000000000000000000C2
:1092AC0000000000000000000000000000000000B2
:1092BC0000000000000000000000000000000000A2
:1092CC00430000000000000000000000000000004F
:1092DC000000000000000000000000000000000082
:1092EC00430000000000000000000000000000002F
:1092FC000000000000000000000000000000000062
:10930C00430000000000000000000000000000000E
:10931C000000000000000000000000000000000041
:10932C0043000000000000000000000000000000EE
:10933C000000000000000000000000000000000021
:10934C0043000000000000000000000000000000CE
:10935C000000000000000000000000000000000001
:10936C0043000000000000000000000000000000AE
:10937C0000000000000000000000000000000000E1
:10938C00430000000000000000000000000000008E
:10939C0000000000000000000000000000000000C1
:1093AC00E98A00104987001000000000AE90001000
:1093BC00AC900010AD900010AD900010AD9000106E
:1093CC00AD900010AD900010AD900010AD9000105D
:1093DC00AD900010AD900010FFFFFFFFFFFFFFFFEF
:1093EC00FFFFFFFFFFFF000001004153434949000D
:1093FC000000000000000000000000000000000061
:10940C0000000000000000000000415343494900E7
:10941C000000000000000000000000000000000040
:10942C00000000000000000000000000A904001073
:10943C0081040010024A1368002BFCDB7047C04605
:10944C000001264010B54378FF2B0BD1032000F010
:10945C0067F9C3685A6801231168194311601168D0
:10946C001942FCD110BD80B230B5C00020D0114BD8
:10947C0007221C682300BA331B885A43236AD3186B
:10948C0019680029FCDA3E210B4B062519600B4BA1
:10949C000B491960A3210B4BC9005D500A49585068
:1094AC005858206A1218002050605A58002AFCDACA
:1094BC0030BDC046F80A02080401264008012640C7
:1094CC001E1F0000000026401C050000F7B5009090
:1094DC000020019100F024F93E4D06002B681A0083
:1094EC005033BC3214681B780419002B5AD000F08E
:1094FC0007F9070003281BD000F0DAF8364A374B7F
:10950C000500D358002B3EDA354A0121300000F01B
:10951C00BFF8002837D10198FFF7A5FF009B002B5F
:10952C003ED02368002BFCDB00F0DAF804002BE0C3
:10953C00062000F0F5F82B68BC331B68C0180368D4
:10954C00002B02DA274C2000FEBD002000F0A8F80A
:10955C00254B9842F6D00023244A190012680120AA
:10956C0000F0D6F80025A842ECD1002000F098F8C5
:10957C001D4A1F4B904203D09D42E3D00135F4E7C6
:10958C009D42B9D1DEE7174C032F05D101210020F4
:10959C0000F0AEF80028F9D1280000F099F8D2E7D5
:1095AC00144CF1E700F084F80D4A0500012130005D
:1095BC0000F06EF8002809D1009B002B08D023681E
:1095CC00002BFCDB00F08CF80400E5E7054CE3E72E
:1095DC00084CE1E7F80A0208000026401C050000D0
:1095EC00280602080500520001018800380602080E
:1095FC00F0490200010050001A4BF7B51B681A4ADB
:10960C005C68042311690B431361012828D030BF17
:10961C002300FC335B6F002B21D100F051F8A32009
:10962C00124B1349134AC0000F681E581568019558
:10963C00114D0D6006251D503E2010600F483E3523
:10964C001D501D58002DFCDA0120FC3460670F60A2
:10965C00A321C9005E50019B136000F011F8F7BD07
:10966C0020BFD5E7F80A020800ED00E00000264014
:10967C0008012640040126401E1F00001C050000A6
:10968C0001B40248844601BC604700BF8B510010F6
:10969C0001B40248844601BC604700BF3D21001064
:1096AC0001B40248844601BC604700BF8924001005
:1096BC0001B40248844601BC604700BFDB040010C3
:1096CC0001B40248844601BC604700BF89510010B8
:1096DC0001B40248844601BC604700BFE30400109B
:1096EC0001B40248844601BC604700BFE51F00106E
:1096FC0001B40248844601BC604700BF1524001029
:10970C0001B40248844601BC604700BF9D72001042
:10971C0001B40248844601BC604700BF59220010C6
:10972C0001B40248844601BC604700BF211F0010F1
:04000005100004EBF8
:00000001FF
